:020000040800F2
:1000000000070020F5040008FD2F0008B52F0008A8
:10001000DD2F0008B52F0008D52F0008F7040008D1
:10002000F7040008F7040008F7040008F13F00088F
:10003000F7040008F7040008F7040008F7040008B4
:10004000F7040008F7040008F7040008F7040008A4
:10005000F7040008F7040008C5650008ED6500080E
:10006000156600083D66000865660008F70400088C
:10007000F7040008F7040008F7040008F704000874
:10008000F7040008F7040008F7040008452F0008EB
:10009000552F0008692F0008F70400088D66000836
:1000A000F7040008F7040008F7040008F704000844
:1000B00061670008F7040008F7040008F704000867
:1000C000F7040008F7040008F7040008F704000824
:1000D000F7040008F7040008F7040008F704000814
:1000E000F1660008F7040008F7040008F7040008A8
:1000F000F7040008F7040008F7040008F7040008F4
:10010000F7040008F7040008F7040008F7040008E3
:10011000F7040008F7040008F7040008F7040008D3
:10012000F7040008F7040008F7040008F7040008C3
:10013000F7040008F7040008F70400087D2F000802
:100140008D2F0008A12F0008F7040008B95B0008F4
:10015000F7040008F7040008F7040008F704000893
:10016000F7040008F7040008F7040008F704000883
:10017000F7040008F7040008F7040008F704000873
:10018000F7040008F7040008F7040008F704000863
:10019000F7040008F7040008F7040008F704000853
:1001A000F7040008F7040008F7040008F704000843
:1001B000F7040008F7040008F7040008F704000833
:1001C000F7040008F7040008F7040008F704000823
:1001D000F7040008F7040008F7040008F704000813
:1001E000D11800080000000000000000000000001E
:1001F00053B94AB9002908BF00281CBF4FF0FF318E
:100200004FF0FF3000F074B9ADF1080C6DE904CE89
:1002100000F006F8DDF804E0DDE9022304B07047E1
:100220002DE9F047089D04468E46002B4DD18A42A9
:10023000944669D9B2FA82F252B101FA02F3C2F1DC
:10024000200120FA01F10CFA02FC41EA030E94406D
:100250004FEA1C48210CBEFBF8F61FFA8CF708FB8E
:1002600016E341EA034306FB07F199420AD91CEB66
:10027000030306F1FF3080F01F81994240F21C8198
:10028000023E63445B1AA4B2B3FBF8F008FB1033E0
:1002900044EA034400FB07F7A7420AD91CEB040415
:1002A00000F1FF3380F00A81A74240F207816444E5
:1002B000023840EA0640E41B00261DB1D44000236A
:1002C000C5E900433146BDE8F0878B4209D9002DCE
:1002D00000F0EF800026C5E9000130463146BDE858
:1002E000F087B3FA83F6002E4AD18B4202D38242C2
:1002F00000F2F980841A61EB030301209E46002D71
:10030000E0D0C5E9004EDDE702B9FFDEB2FA82F2C5
:10031000002A40F09280A1EB0C014FEA1C471FFA23
:100320008CFE0126200CB1FBF7F307FB131140EA0A
:1003300001410EFB03F0884208D91CEB010103F1D7
:10034000FF3802D2884200F2CB804346091AA4B299
:10035000B1FBF7F007FB101144EA01440EFB00FE6D
:10036000A64508D91CEB040400F1FF3102D2A645D2
:1003700000F2BB800846A4EB0E0440EA03409CE771
:10038000C6F12007B34022FA07FC4CEA030C20FA1E
:1003900007F401FA06F31C43F9404FEA1C4900FA3E
:1003A00006F3B1FBF9F8200C1FFA8CFE09FB1811BB
:1003B00040EA014108FB0EF0884202FA06F20BD92E
:1003C0001CEB010108F1FF3A80F08880884240F27E
:1003D0008580A8F102086144091AA4B2B1FBF9F0C2
:1003E00009FB101144EA014100FB0EFE8E4508D9BD
:1003F0001CEB010100F1FF346CD28E456AD9023842
:10040000614440EA0840A0FB0294A1EB0E01A14226
:10041000C846A64656D353D05DB1B3EB080261EB94
:100420000E0101FA07F722FA06F3F1401F43C5E96E
:10043000007100263146BDE8F087C2F12003D840A4
:100440000CFA02FC21FA03F3914001434FEA1C47E6
:100450001FFA8CFEB3FBF7F007FB10360B0C43EAD8
:10046000064300FB0EF69E4204FA02F408D91CEB88
:10047000030300F1FF382FD29E422DD90238634486
:100480009B1B89B2B3FBF7F607FB163341EA034126
:1004900006FB0EF38B4208D91CEB010106F1FF3875
:1004A00016D28B4214D9023E6144C91A46EA00466C
:1004B00038E72E46284605E70646E3E61846F8E6FE
:1004C0004B45A9D2B9EB020864EB0C0E0138A3E747
:1004D0004646EAE7204694E74046D1E7D0467BE728
:1004E000023B614432E7304609E76444023842E7A0
:1004F000704700BF02E000F000F8FEE772B6374830
:1005000080F30888364880F3098836483649086001
:1005100040F20000CCF200004EF63471CEF2000141
:100520000860BFF34F8FBFF36F8F40F20000C0F23F
:10053000F0004EF68851CEF200010860BFF34F8FF5
:10054000BFF36F8F4FF00000E1EE100A4EF63C71E2
:10055000CEF200010860062080F31488BFF36F8F8D
:1005600004F0F2FF05F0D6FE4FF055301F491B4A4C
:1005700091423CBF41F8040BFAE71D49184A9142E9
:100580003CBF41F8040BFAE71A491B4A1B4B9A423D
:100590003EBF51F8040B42F8040BF8E7002018495D
:1005A000184A91423CBF41F8040BFAE704F0D0FF2F
:1005B00005F004FF144C154DAC4203DA54F8041B4B
:1005C0008847F9E700F042F8114C124DAC4203DACB
:1005D00054F8041B8847F9E704F0B8BF000700206F
:1005E000002300200000000808ED00E000010020CA
:1005F00000070020486D000800230020B0230020E1
:10060000B023002008670020E0010008E401000892
:10061000E4010008E40100082DE9F04F2DED108AF7
:10062000C1F80CD0C3689D46BDEC108ABDE8F08FC0
:10063000002383F311882846A047002004F090FA95
:10064000FEE704F0E9F900DFFEE70000F8B501F08D
:1006500055F904F013FF074604F062FF0546B8BBE6
:10066000204B9F4234D001339F4234D01E4B27F0A1
:10067000FF029A4232D1F8B200F036FF2E4642F223
:10068000107400F037FF08B10024264601F038FD51
:1006900020B1032000F07CF80024264635B1134B2E
:1006A0009F4203D004F034FF00242646002004F0CB
:1006B000EFFE0EB100F082F801F0D2FA00F086FFF2
:1006C00001F082F9204600F0DFF800F077F8F9E752
:1006D0002E460024D5E704460126D2E7064641F21D
:1006E0008834CEE7010007B0000008B0263A09B010
:1006F00008B501F03BF9A0F120035842584108BD6C
:1007000007B541F21203022101A8ADF8043001F04F
:100710004BF903B05DF804FB38B5302383F311883F
:10072000174803680BB104F0E7FA164A144800238F
:100730004FF47A7104F0D6FA002383F31188124C37
:10074000236813B12368013B2360636813B16368B6
:10075000013B63600D4D2B7833B963687BB9022090
:1007600001F0F8F9322363602B78032B07D163681B
:100770002BB9022001F0EEF94FF47A73636038BDB3
:10078000B023002019070008D0240020C82300202F
:10079000084B187003280CD8DFE800F008050208A1
:1007A000022001F0CDB9022001F0C0B9024B0022B5
:1007B0005A607047C8230020D024002010B501F0F3
:1007C0009FFC30B1294B03221A70294B00225A603A
:1007D00010BD284B284A1C4619680131F8D0043353
:1007E0009342F9D16268254B9A42F1D9244B9B6818
:1007F00003F1006303F580339A42E9D204F05CFE12
:1008000004F06EFE002001F0F9F80220FFF7C0FFAF
:100810001C4B1A6C00221A64196E1A66196E596CF8
:100820005A64596E5A665A6E5A6942F080025A6189
:100830005A6922F080025A615A691A6942F00052DC
:100840001A611A6922F000521A611B6972B64FF0E0
:10085000E0233021C3F8084DD4E9003281F3118838
:100860009D4683F308881047B2E700BFC8230020E5
:10087000D02400200000010820000108FFFF00082C
:1008800000230020003802402DE9F04F93B0AC4B1C
:1008900000902022FF210AA89D6801F08BF9A94A47
:1008A0001378A3B9A848012103601170302383F3A2
:1008B000118803680BB104F01FFAA44AA248002370
:1008C0004FF47A7104F00EFA002383F31188009B31
:1008D00013B19F4B009A1A609E4A009C1378032B19
:1008E0001EBF002313709A4A4FF0000A18BF5360CE
:1008F000D3465646D146012001F022F924B1944B4B
:100900001B68002B00F01582002001F02FF80390E7
:10091000039B002B01DA00F0ABFE039B002BEDDB09
:10092000012001F003F9039B213B162BE3D801A220
:1009300052F823F091090008B90900084D0A00088F
:10094000F7080008F7080008F7080008D70A0008A9
:10095000A70C0008C10B0008230C00084B0C000872
:10096000710C0008F7080008830C0008F70800085D
:10097000F50C0008310A0008F7080008390D0008D6
:100980009D090008310A0008F7080008230C000838
:100990000220FFF7ADFE002840F0F581009B022108
:1009A000BAF1000F08BF1C4605A841F21233ADF89A
:1009B000143000F0F9FF9EE74FF47A7000F0D6FF94
:1009C000071EEBDB0220FFF793FE0028E6D0013F75
:1009D000052F00F2DA81DFE807F0030A0D10133665
:1009E00005230593042105A800F0DEFF17E0544815
:1009F0000421F9E758480421F6E758480421F3E7B1
:100A00004FF01C08404600F0FBFF08F10408059079
:100A1000042105A800F0C8FFB8F12C0FF2D1012085
:100A200000FA07F747EA0B0B5FFA8BFB4FF0000960
:100A300001F00CF926B10BF00B030B2B08BF0024BF
:100A4000FFF75EFE57E746480421CDE7002EA5D00C
:100A50000BF00B030B2BA1D10220FFF749FE074639
:100A600000289BD0012000F0C9FF0220FFF790FE74
:100A700000261FFA86F8404600F0D0FF044690B1E9
:100A80000021404600F0E2FF01360028F1D1BA46CD
:100A9000044641F21213022105A8ADF814303E4677
:100AA00000F082FF27E70120FFF772FE2546244B66
:100AB0009B68AB4207D9284600F0A2FF013040F006
:100AC00067810435F3E7234B00251D70204BBA46A0
:100AD0005D603E46ACE7002E3FF460AF0BF00B03C9
:100AE0000B2B7FF45BAF0220FFF752FE322000F0A9
:100AF0003DFFB0F10008FFF651AF18F003077FF497
:100B00004DAF0F4A926808EB050393423FF646AF9C
:100B1000B8F5807F3FF742AF124B0193B84523DD14
:100B20004FF47A7000F022FF0390039A002AFFF638
:100B300035AF019B039A03F8012B0137EDE700BFA6
:100B400000230020CC240020B02300201907000837
:100B5000D0240020C82300200423002008230020E4
:100B60000C230020CC230020C820FFF7C1FD07463E
:100B700000283FF413AF1F2D11D8C5F120024245C4
:100B80000AAB25F0030028BF42468349019218446E
:100B900000F0EAFF019A8048FF2101F00BF84FEACC
:100BA000A8037D490193C8F38702284601F00AF89B
:100BB000064600283FF46DAF019B05EB830537E740
:100BC0000220FFF795FD00283FF4E8AE00F05EFF3D
:100BD00000283FF4E3AE0027B846704B9B68BB4249
:100BE00018D91F2F11D80A9B01330ED027F0030309
:100BF00012AA134453F8203C05934046042205A949
:100C000001F036FA04378046E7E7384600F0F8FE90
:100C10000590F2E7CDF81480042105A800F0C4FE89
:100C200006E70023642104A8049300F0B3FE002823
:100C30007FF4B4AE0220FFF75BFD00283FF4AEAEB8
:100C4000049800F00BFF0590E6E70023642104A858
:100C5000049300F09FFE00287FF4A0AE0220FFF76F
:100C600047FD00283FF49AAE049800F007FFEAE73A
:100C70000220FFF73DFD00283FF490AE00F016FF84
:100C8000E1E70220FFF734FD00283FF487AE05A915
:100C9000142000F011FF04210746049004A800F07E
:100CA00083FE3946B9E7322000F060FE071EFFF6EA
:100CB00075AEBB077FF472AE384A926807EB090342
:100CC00093423FF66BAE0220FFF712FD00283FF47F
:100CD00065AE27F003074F44B9453FF4A9AE484637
:100CE00000F08EFE0421059005A800F05DFE09F1DC
:100CF0000409F1E74FF47A70FFF7FAFC00283FF49B
:100D00004DAE00F0C3FE002844D00A9B01330BD047
:100D100008220AA9002000F055FF00283AD020221E
:100D2000FF210AA800F046FFFFF7EAFC1C4803F089
:100D30001DFF13B0BDE8F08F002E3FF42FAE0BF077
:100D40000B030B2B7FF42AAE0023642105A8059327
:100D500000F020FE074600287FF420AE0220FFF7B7
:100D6000C7FC804600283FF419AEFFF7C9FC41F2EA
:100D7000883003F0FBFE059800F09AFF464600F02D
:100D800065FF3C46B7E5064652E64FF0000905E62A
:100D9000BA467EE637467CE6CC23002000230020BE
:100DA000A0860100094A136849F2690099B21B0C38
:100DB00000FB01331360064B186844F2506182B2A5
:100DC000000C01FB0200186080B27047182300205D
:100DD0001423002010B500211022044600F0EAFE82
:100DE000034B03CB206061601868A06010BD00BF9A
:100DF000107AFF1F2DE9F041ADF54C7D0DF12C0867
:100E00006AAC40F2751207460D460CA80021C8F8DE
:100E1000001000F0CFFE4FF4C4720021204600F015
:100E2000C9FE02F0F3F8274B4FF47A72B0FBF2F0F0
:100E3000186093E80700022384E807000DF5E570C9
:100E40002382FFF7C7FF47F217031F49238407A830
:100E500005F096FD0F2384F832310DF2DB2207AB4B
:100E60000DF1240C1E4603CE6645106051603346DA
:100E700002F10802F6D130681060B188B37993713D
:100E8000918020464146012200F014FF0023039385
:100E9000AB7E029305F11903019380B20123CDE9E2
:100EA00004800093E97E05A3D3E90023384602F0CD
:100EB00075FC0DF54C7DBDE8F08100BF9E6AC42134
:100EC000818A46EED8240020906900082DE9F0417F
:100ED0002C4C237ADAB080460D465BBB27A9284606
:100EE00000F0F8FF0746002842D19DF89D60C82E0B
:100EF0003ED801464FF4A662204600F05BFE4FF458
:100F00008073C4F8F8314FF40073C4F80C334FF415
:100F10004073C4F8203432460DF19E0104F10900FB
:100F200000F022FE26449DF89C30777223720BB9A4
:100F3000EB7E23728122002106AC27A800F03AFE46
:100F40000122214627A801F001F800230393AB7E7C
:100F5000029305F1190380B201932823CDE90440DF
:100F60000093E97E05A3D3E90023404602F016FC76
:100F70005AB0BDE8F08100BFAFF300802641727225
:100F8000DF25D7B7C0560020F0B5254E4FF48A753F
:100F900005FB0065F1B096F8D83085F8DC30002408
:100FA000D822214685F8E8403AA800F003FE06F171
:100FB000090000F0F7FDD5F8E4308DF8F000C2B27A
:100FC00006AF06F109010DF1F100CDE93A3400F068
:100FD000CBFD394601223AA800F0E4FF80B2CDE90A
:100FE000047008230127CDE9023706F1D8030193E5
:100FF00030230093317A0B4807A3D3E9002302F092
:10100000CDFBA04206DD02F001F8C5F8E00038464D
:1010100071B0F0BD2046FBE778F6339F93CACD8DC3
:10102000C0560020F03400202DE9F04F274FDFF8A4
:10103000A880274E87B0384602F0DCFB0346002824
:101040003DD00024CDE90344ADF81440027B8DF877
:10105000142099684068029403AA03C21B681D4DBE
:1010600043F000430293A146A2462B68D3F810B088
:1010700001F0CEFF10EB080241F100032846CDF845
:1010800000A002A9D84704F2344440F668030028BF
:10109000C8BF49F0010905F586559C4205F11005C8
:1010A000E3D1B9F1000F05D0384602F0A7FB86F86E
:1010B00000A0C0E73378072B04D80133337007B0A2
:1010C000BDE8F08F014802F099FBF8E7F03400200A
:1010D000F55B00202035002040420F0070B50D4622
:1010E00014461E4602F0B6FA50B9022E10D1012C59
:1010F0000ED112A3D3E90023C5E90023012007E0A4
:10110000282C10D005D8012C09D0052C0FD0002098
:1011100070BD302CFBD10BA3D3E90023ECE70BA36C
:10112000D3E90023E8E70BA3D3E90023E4E70BA30B
:10113000D3E90023E0E700BFAFF30080401DA1200A
:1011400026812A0B78F6339F93CACD8D9E6AC421DF
:10115000818A46EE26417272DF25D7B7F017304AF2
:1011600039059E5638B505460E4C0021013500F074
:101170006DFCA4F82C55B4F82C0500F04FFC78B1A8
:10118000B4F82C0500F05AFC014648B9B4F82C0517
:1011900000F05CFCB4F82C350133A4F82C35EAE7F8
:1011A00038BD00BFC0560020F8B50E4C0E4F0226C9
:1011B000A4F5805343F8487C237E3BB965692DB183
:1011C000284601F01BF8284605F01AFB204601F0DE
:1011D00015F8A4F58654012EA4F1100400D1F8BD31
:1011E0000126E5E7385600204C6A00082DE9F04F4B
:1011F0008FB000AF05460C4602F02CFA002849D10A
:10120000237E022B1BD1E38A012B18D101F0FEFEB5
:101210000646FFF7C7FD03464FF4C870DFF8C482E7
:10122000B3FBF0F206F5167602FB103316FA83F3E1
:10123000C8F80030E37E33B9A34B00221A703C3764
:10124000BD46BDE8F08F07F12401204600F000FE06
:101250000028F4D107F11400FFF7BCFD97F82640F1
:1012600007F11401224607F1270005F013FB0028BF
:10127000E2D10F2C08D8944B1C70D8F80030A3F59D
:101280001673C8F80030DAE797F82410284602F001
:10129000D9F9D4E7E38A282B2BD010D8012B23D0FF
:1012A000052BCCD1BFF34F8F8849894BCA6802F414
:1012B000E0621343CB60BFF34F8F00BFFDE7302BDD
:1012C000BDD1844EE17E327A9142B8D1607E314602
:1012D000002291F8DC50854200F0A5800132042AFA
:1012E00001F58A71F5D1AAE721462846FFF782FD6C
:1012F000A5E721462846FFF7E9FDA0E7B2F8EC5044
:101300007B6005F103094FEA99094FEA8902D11D73
:10131000C908A8EBC1039D46EB460021584600F0E2
:1013200049FC04F1EE012A463144584600F01CFC09
:101330007B6813B9012000F061FB96F8D20000F041
:101340006DFB044630B9307200F0A0FB204600F07F
:1013500055FBB1E0D6F8D4203AB996F8D200B6F8E9
:101360002C25824201D8FFF7FDFED6F8D4202A446E
:10137000944208D296F8D200B6F82C250130824269
:1013800001D8FFF7EFFE70685FFA89F2594600F066
:1013900019FC08B9C54679E0726896F8D2002A446B
:1013A0007260D6F8D42005EB0209C6F8D49000F09C
:1013B00035FB814509D396F8D220D6F8D400013206
:1013C000001B86F8D220C6F8D400FF2D0FD80024C9
:1013D000347200F05BFB204600F010FB00F090FE42
:1013E0003D4B188108B9FFF7E9F9C54627E7BB6807
:1013F00096F8D9000AFB0362FB68D2F8E41082F881
:10140000E83001F58061C2F8E030C2F8E410FFF77F
:10141000BBFDFFF709FE96F8D920013202F0030266
:1014200086F8D920B6E74FF48A7A0AFB02F505F16F
:10143000EA013144204600F0E1FDF86000287FF425
:10144000FEAE3544012285F8E82001F0DFFDD5F835
:10145000E020D6ED007ADFED216A801A192838BF26
:10146000192040F6B832904228BF1046B8EE677A8D
:1014700007EE900AF8EEE77A67EEA67ADFED186AD3
:10148000E7EE267AFCEEE77AC6ED007A96F8D930D8
:10149000BB60BA6873680AFB02F4321992F8E8106C
:1014A00059B1D2F8E4108B42E8463FF427AF00214F
:1014B00082F8E810C2F8E010C5467368064A9B0A35
:1014C00001331381BBE600BFE934002000ED00E0EA
:1014D0000400FA05C0560020D8240020CDCCCC3D15
:1014E0006666663FEC340020014B1870704700BF01
:1014F000E424002030B54FF000542B4B22689A4270
:1015000085B007D004F016F8044620BB002420461E
:1015100005B030BD254B627D25481A70237D0372CE
:101520004FF48073C0F8F8314FF40073C0F80C33F7
:1015300000254FF44073C0F820341E49C0F8E45031
:10154000C922093000F010FB2046E022294600F0B5
:1015500031FB0124DBE7184A184D136C43F000738C
:101560001364AA6D164B9A42D0D12B6E013B7E2B91
:10157000CCD8144A07CA01AB83E8070018460321F8
:1015800000F08CFD6B6D83424FF00003BED12A6DDD
:101590008A4201BFAB65054B2A6E1A7003BF0A4B26
:1015A000EA6D1A601C46B2E79AAD44C5E4240020F7
:1015B000C05600201600002000380240006600409F
:1015C0005041A0B0586600401023002037B500F00D
:1015D00097FD1D4D1D4C2881022321681C486B710D
:1015E000012201F097FB1B48216850F8D03F0122EF
:1015F0005B68984700230193174B184900931848DC
:10160000184B4FF4805201F0F5FF174B197811B1C8
:10161000134802F017F801F0F9FC0446FFF7C2FB8B
:101620004FF4C873B0FBF3F202FB130304F516701A
:1016300010FA83F00D4B186003F072FF08B10F230E
:101640002B8103B030BD00BFD82400201023002020
:101650002035002020450020DD100008E82400206F
:10166000F0340020ED110008E4240020EC340020C8
:101670002DE9F04F2DED028BDFF8508293B00BAFC8
:101680009FED838BFFF7D0FC00230A93ADF8343035
:101690000B937B600025844CDFF810A22E460123BB
:1016A0008DF81C3023688DED008B4FF0000BD3F8C4
:1016B00008908DF81DB05B460DF11D0207A920466C
:1016C000C8479DF81C90B9F1000F24D0D8F8143009
:1016D00083F48073C8F81430102259460EA800F025
:1016E00069FA236808AA5E690AA90DF11E0320465B
:1016F000B04797E803000FAB83E803009DF8343050
:101700008DF844300A9B0E930EA9DDE9082350465C
:1017100002F052FA4E4605F2344540F6680304F5ED
:1017200086549D4204F11004B9D1002EB2D15F4815
:1017300001F090FF002840D15D4D01F067FC2B685F
:1017400098423AD301F062FC0446FFF72BFB4FF4BA
:10175000C873B0FBF3F202FB130304F5167010FA22
:1017600083F02860534D8DF828602E7816B9012338
:101770008DF82830C6F11004E4B20EA8FFF72AFB5A
:10178000062C28BF06240EAB224699190DF129001C
:1017900000F0EAF90AAB0393182302930134464B95
:1017A0000193E4B201230093404804943AA3D3E99F
:1017B000002301F095FF00232B7001F027FC3F4A26
:1017C0003F4C1368C31AB3F57A7F2FD3106001F032
:1017D0001FFC02460B46354802F01AF8334801F068
:1017E00039FF18B3237A374D002B14BF032302238C
:1017F0006B7101F00BFC0EAE4FF47A730122B0FB5B
:10180000F3F031462860284600F0FAFA18230293D4
:101810002D4B019380B240F25513CDE90360009344
:1018200022481FA3D3E9002301F05AFF237A93B182
:1018300001F0ECFB002506464FF48A7794F8D900B6
:10184000284400F0030007FB004393F8E82072B13E
:101850000135042DF2D1C82003F088F9237A002B3A
:101860007FF40DAF13B0BDEC028BBDE8F08FD3F861
:10187000E02042B12368FA2B38BFFA23B21A0533AD
:10188000B2EB430FE4D3FFF77FFB0028E0D1E2E7A0
:101890000000000000000000401DA12026812A0B4E
:1018A000F1C6A7C1D068080F20350020F034002011
:1018B000EC340020E9340020E8340020F05B002004
:1018C000C0560020D8240020F45B0020000802400D
:1018D00008B5064800F094FF054800F091FFBDE808
:1018E0000840044A0449002004F084BF2035002049
:1018F000F0450020345C0020A9110008704700006A
:1019000070B50F4B1B780133DBB2012B0C4611D89D
:101910000C4D29684FF47A730E6AA2FB033201461C
:1019200022462846B047844204D1074B00221A7051
:10193000012070BD4FF4FA7003F018F90020F8E7A9
:101940001C230020A85E0020245C002070B5044603
:101950004FF47A76412C254628BF412506FB05F039
:1019600003F004F9641BF5D170BD000007B5002336
:10197000024601210DF107008DF80730FFF7C0FF87
:1019800020B19DF8070003B05DF804FB4FF0FF3075
:10199000F9E700000A4608B50421FFF7B1FF80F01F
:1019A0000100C0B2404208BD30B4054C2368DD6977
:1019B000044B0A46AC460146204630BC604700BF97
:1019C000A85E0020A086010070B503F0EFFB094E71
:1019D000094D3080002428683388834208D903F0F9
:1019E000DFFB2B6804440133B4F5803F2B60F2D356
:1019F00070BD00BF265C0020F85B002003F086BCB1
:101A000000F1006000F580300068704700F1006070
:101A1000920000F5803003F00FBC0000054B1A68FF
:101A2000054B1B889B1A834202D9104403F0B8BBB4
:101A300000207047F85B0020265C0020024B1B68EA
:101A4000184403F0B5BB00BFF85B0020024B1B68D5
:101A5000184403F0C5BB00BFF85B002010F003037F
:101A60000AD1B0F5047F05D200F10050A0F5104076
:101A7000D0F80038184670470023FBE700F100500B
:101A8000A0F51040D0F8100A70470000064991F800
:101A9000243033B10023086A81F824300822FFF78C
:101AA000B5BF0120704700BFFC5B0020014B1868E8
:101AB000704700BF002004E070B5194B1D68194B3A
:101AC0000138C5F30B0408442D0C04221E88A642DD
:101AD0000BD15C680A46013C824213460FD214F9CE
:101AE000016F4EB102F8016BF6E7013A03F108030A
:101AF000ECD181420B4602D22C2203F8012B0A4A78
:101B000005241688AE4204D1984284BF967803F823
:101B1000016B013C02F10402F3D1581A70BD00BF01
:101B2000002004E0E0690008CC690008022802BF38
:101B3000024B4FF480729A61704700BF0008024068
:101B4000022802BF024B4FF080729A61704700BFBB
:101B500000080240022801BF024A536983F48073DF
:101B6000536170470008024010B50023934203D030
:101B7000CC5CC4540133F9E710BD000010B5013846
:101B800010F9013F3BB191F900409C4203D11AB1D9
:101B90000131013AF4E71AB191F90020981A10BD09
:101BA0001046FCE703460246D01A12F9011B002931
:101BB000FAD1704702440346934202D003F8011B56
:101BC000FAE770472DE9F8431F4D144695F8242095
:101BD0000746884652BBDFF870909CB395F82430D6
:101BE0002BB92022FF2148462F62FFF7E3FF95F82B
:101BF0002400C0F10802A24228BF2246D6B24146C4
:101C0000920005EB8000FFF7AFFF95F82430A41B8E
:101C10001E44F6B2082E17449044E4B285F82460BE
:101C2000DBD1FFF733FF0028D7D108E02B6A03EBA5
:101C300082038342CFD0FFF729FF0028CBD10020B9
:101C4000BDE8F8830120FBE7FC5B0020024B1A781B
:101C5000024B1A70704700BF245C00201C23002038
:101C600010B5104C104802F0B1FA21460E4802F0AF
:101C7000D9FA2468626DD2F8043843F00203C2F83E
:101C800004384FF47A70FFF761FE0849204602F0ED
:101C9000CFFB626DD2F8043823F00203C2F8043897
:101CA00010BD00BF386B0008A85E0020406B000824
:101CB000704700002DE9F0470D460446002190468C
:101CC000284640F27912FFF775FF234620220021B3
:101CD000284601F013FF231D02222021284601F08F
:101CE0000DFF631D03222221284601F007FFA31DDB
:101CF00003222521284601F001FF04F108031022E8
:101D00002821284601F0FAFE04F1100308223821A8
:101D1000284601F0F3FE04F1110308224021284671
:101D200001F0ECFE04F1120308224821284601F0DC
:101D3000E5FE04F1140320225021284601F0DEFEC6
:101D400004F1180340227021284601F0D7FE04F167
:101D500020030822B021284601F0D0FE04F121031F
:101D60000822B821284601F0C9FE04F12207C02646
:101D70003B46314608222846083601F0BFFEB6F53C
:101D8000A07F07F10107F3D104F1320308223146A5
:101D9000284601F0B3FE002704F1330A94F83230EC
:101DA0004FEAC7099F4209F5A47615D3B8F1000F91
:101DB00008D1314604F599730722284601F09EFEAA
:101DC00009F24F16274694F832213B1B93420CD35D
:101DD000F01DC008BDE8F0870AEB07030822314672
:101DE000284601F08BFE0137D8E707F2331331465E
:101DF0000822284601F082FE08360137E3E700009A
:101E000013B504460846002101602346C0F80310BC
:101E10002022019001F072FE0198231D0222202150
:101E200001F06CFE0198631D0322222101F066FE81
:101E30000198A31D0322252101F060FE019804F101
:101E400008031022282101F059FE072002B010BD1E
:101E5000F7B50023047F00910E4607221946054678
:101E600001F010FD731C0093012200230721284676
:101E700001F008FDC4B9B31C0093052223460821D4
:101E8000284601F0FFFC0D243746B278BB1B934275
:101E900011D32B7FA88A0734E408BBB9844294BFCE
:101EA0000020012003B0F0BDAB8ADB00083BDB085B
:101EB000B3700824E8E7FB1C0093214600230822A6
:101EC000284601F0DFFC08340137DEE7201A18BF8E
:101ED0000120E7E7F7B50023047F00910E460822B2
:101EE0001946054601F0CEFC731CC4B908220093C4
:101EF00011462346284601F0C5FC102401237278C0
:101F00005F1C013B934211D32B7FA88A0734E4085E
:101F1000BBB9844294BF0020012003B0F0BDAB8A5E
:101F2000DB00083BDB0873700824E7E7F319009334
:101F3000214600230822284601F0A4FC08343B4631
:101F4000DDE7201A18BF0120E7E70000F8B50E46CC
:101F500005461446002181223046FFF72BFE2B4612
:101F600008220021304601F0C9FD7CB96B1C072214
:101F70000821304601F0C2FD0F2401236A785F1C5E
:101F8000013B934204D3E01DC008F8BD0824F4E7E8
:101F9000EB1921460822304601F0B0FD08343B46DB
:101FA000ECE70000F8B50E46054614460021CE22A7
:101FB0003046FFF7FFFD2B4628220021304601F076
:101FC0009DFD7CB905F1080308222821304601F067
:101FD00095FD30242F462A7A7B1B934204D3E01DC3
:101FE000C008F8BD2824F5E707F1090321460822B7
:101FF000304601F083FD08340137ECE7F7B5047F84
:1020000000910E46012310220021054601F03AFC02
:10201000C4B9B31C0093092223461021284601F0BD
:1020200031FC192437467288BB1B9A4211D82B7F8A
:10203000A88A0734E408BBB9844294BF0020012079
:1020400003B0F0BDAB8ADB00103BDB0873801024CB
:10205000E8E73B1D0093214600230822284601F0B3
:1020600011FC08340137DEE7201A18BF0120E7E72A
:1020700030B5094D0A4491420DD011F8013B58404A
:10208000082340F30004013B2C4013F0FF0384EAD3
:102090005000F6D1EFE730BD2083B8EDF7B54FF033
:1020A000FF33DFF854C0DFF854E000EB81011A463B
:1020B00088421CD050F8044B019401AF042417F857
:1020C000015B82EA05620825DB18164605F1FF353B
:1020D0005241002EBCBF83EA0C0382EA0E0215F0C7
:1020E000FF05F1D1013C14F0FF04E8D1E0E7D8434B
:1020F000D14303B0F0BD00BF9336EAA9EBE1F04253
:10210000F7B5384A106851686B4603C36A463649CA
:102110003648082304F0CEFB0446002833D10A25B4
:10212000334A106851686B4603C36A4631492F48E9
:10213000082304F0BFFB0446002849D00369B3F527
:10214000E02F45D8B0F8661041F2707291423FD14D
:10215000294A024402F15C018B4239D35C3B23499A
:1021600000209E1AFFF784FF3246074604F16401FF
:102170000020FFF77DFFA3689F4229D1E3689842C2
:1021800008BF002524E00369B3F5E02F27D8418B71
:1021900041F27072914220D1174A024402F11001BB
:1021A0008B4218D3103B114900209D1AFFF760FFA6
:1021B0002A46064604F118010020FFF759FFA368DC
:1021C0009E4202D1E368984201D00D25A8E7002580
:1021D000284603B0F0BD1025A2E70C25A0E70B258B
:1021E0009EE700BF006A0008DCFF0600000001084F
:1021F000096A000890FF06000800FFF710B5037C8D
:10220000044613B9006804F03DFB204610BD0000F1
:102210000023BFF35B8FC360BFF35B8FBFF35B8FA4
:102220008360BFF35B8F7047BFF35B8F0068BFF3C2
:102230005B8F704770B505460C30FFF7F5FF05F171
:10224000080604463046FFF7EFFFA04206D93046A5
:102250006D68FFF7E9FF2544281A70BD3046FFF787
:10226000E3FF201AF9E7000070B50546406898B111
:1022700005F10800FFF7D8FF05F10C0604463046CB
:10228000FFF7D2FF8442304694BF6D680025FFF708
:10229000CBFF013C2C44201A70BD000038B50C4621
:1022A0000546FFF7C7FFA04210D305F10800FFF76E
:1022B000BBFF04446868B4FBF0F100FB1144BFF3BA
:1022C0005B8F0120AC60BFF35B8F38BD0020FCE763
:1022D0002DE9F041144607460D46FFF7C5FF84423D
:1022E00028BF0446D4B1B84658F80C6B4046FFF7F7
:1022F0009BFF3044286040467E68FFF795FF331A05
:102300009C4203D86C600120BDE8F0816B60A41B87
:102310003B68AB602044E8600220F5E72046F3E725
:1023200038B50C460546FFF79FFFA04210D305F1D4
:102330000C00FFF779FF04446868B4FBF0F100FB80
:102340001144BFF35B8F0120EC60BFF35B8F38BD9E
:102350000020FCE72DE9FF41884669460746FFF764
:10236000B7FF6C4606B204EBC6060025B44209D09E
:102370006268206808EB0501FFF7F6FB6368083424
:102380001D44F3E729463846FFF7CAFF284604B044
:10239000BDE8F081F8B505460C300F46FFF744FF65
:1023A00005F1080604463046FFF73EFFA0423046DE
:1023B00088BF6C68FFF738FF201A386020B13046BC
:1023C0002C68FFF731FF2044F8BD000073B51446B8
:1023D00006460D46FFF72EFF844228BF04460190B3
:1023E000DCB101A93046FFF7D5FF019B33B9326854
:1023F000C5E90233C5E9002401200CE09C4238BF46
:1024000001942860019868608442F5D93368AB6014
:10241000241AEC60022002B070BD2046FBE70000E9
:102420002DE9FF410F466946FFF7D0FF6C4600B229
:1024300004EBC0050026AC4209D0D4F8048054F85F
:10244000081BB8194246FFF78FFB4644F3E73046B6
:1024500004B0BDE8F081000038B50546FFF7E0FFA5
:10246000044601462846FFF719FF204638BD000004
:10247000302383F3118862B670470000002383F392
:10248000118862B67047000010B4026854681A469A
:1024900023465DF8044B1847012070470020704721
:1024A0000020704770470000002070470E207047E2
:1024B00000F5805090F8C800C0F34000704700005D
:1024C00000F5805090F9C90070470000F7B50C681E
:1024D000BDF8207014F000541E466FD10B7B082B02
:1024E0006CD8FFF7C5FF4569AB685B010CD4AB68DE
:1024F0001B0108D4AC6814F080545DD1FFF7BEFF17
:10250000204603B0F0BD01240B6804F1180C002B29
:10251000B8BFDB004FEA0C1CB4BF43F004035B05FB
:1025200045F80C300B680FFA84FC13F0804F18BF8D
:1025300005EB0C1E05EB0C1C1EBFDEF8803143F0D2
:102540000203CEF880310B7BCCF8843105EB041507
:102550008B68C5F88C314B68C5F88831DCF8803160
:1025600043F00103CCF8803100EB441541F26803DD
:102570001D4403EB44130344C5E9002608330D460C
:1025800001F10C0C55F804EB43F804EB6545F9D167
:1025900084342D881D8000EB441407F00303257953
:1025A00025F00B052B432371FFF768FF0097334697
:1025B00000F04EFD0120A4E70224A5E74FF0FF3014
:1025C0009FE7000013B500F580540191E06DFFF71F
:1025D0004BFE1F280AD90199E06D2022FFF7BAFEB1
:1025E000A0F120035842584102B010BD0020FBE783
:1025F00008B500F58050FFF73BFFC06DFFF708FE00
:10260000BDE80840FFF73ABF0022026082814260C5
:102610008260704710B500220023C0E90023002328
:10262000044603810C30FFF7EFFF204610BD000089
:10263000F0B5054600F580500C4690F8C83013F010
:10264000040FC3F3800108BF114661F3820304F154
:10265000840680F8C83005EB461389B01B79D8078B
:102660002ED57AB319072DD46846FFF7D3FF05EBB3
:10267000441303F5835303F1180703AA10331868B2
:102680005968144603C40833BB422246F7D1186880
:1026900020609B88A380DDE90E23CDE90023012380
:1026A000ADF808302B686946DB6B2846984705EB88
:1026B00046152B791A075CBF43F008032B7101E024
:1026C000002AF4D109B0F0BD2DE9F047074688B0E3
:1026D00007F5805468469A468846FFF7C9FE91463A
:1026E000FFF798FFE06DFFF7A5FD1F2829D9E06DE2
:1026F00020226946FFF7B0FE202822D103AD4446D0
:1027000005AB2E4603CE9E4220606160354604F143
:102710000804F6D130682060B388A380DDE9002387
:10272000C9E90023BDF80830AAF80030FFF7A6FE7B
:102730004A4653464146384608B0BDE8F04700F0E7
:1027400075BCFFF79BFE002008B0BDE8F0870000D5
:102750002DE9F84F0023C0E90133264B044640F829
:10276000183B0F46FFF750FF04F12800FFF752FF18
:1027700004F1480804F582554646083530462036AF
:10278000FFF748FFAE42F9D104F580554FF480536E
:102790004FF00009C5E91339C5F848800123EE65FB
:1027A00004F5875804F58456C5F8549085F85830D8
:1027B00085F86030083608F108084FF0000A4FF03D
:1027C000000B46E908ABA6F11800FFF71DFF203605
:1027D00046F8289C4645F4D1012F85F8C97002D9E6
:1027E000054800F00DFC054B53F827306361204687
:1027F000BDE8F88F4C6A0008146A0008306A0008C7
:1028000010B5044B197804464A1C1A70FFF7A0FF54
:10281000204610BD305C00202DE9F047002950D043
:10282000294B2A4FB7FBF1F599428CBF0A2311239C
:10283000581EB5FBF3FC03FB1C53C4B22BB102289A
:102840000346F5D80020BDE8F0870CF1FF36B6F559
:10285000806FF7D2C4EBC40E0EF103034FEAE30915
:10286000C3F3C703A4EB030809F1010A4FF47A7517
:102870005FFA88F009FB05555AFA88F8B5FBF8F5B8
:10288000B5F5617FC1BF0EF1FF33C3F3C703E01A93
:10289000C0B25C1C50FA84F40CFB04F4B7FBF4F4F3
:1028A000A142CFD1013BDBB20F2BCBD80138C0B254
:1028B0000728C7D80021107116809170D3700120AD
:1028C000C1E70846BFE700BF3F420F0080DE80023D
:1028D00070B505460E464FF47A746B695B6803F079
:1028E0000103B34207D04FF47A7002F03FF9013C84
:1028F000F3D1204670BD0120FCE7000030B54269ED
:10290000936913F0700F16D000230B4C936103F101
:10291000840200EB421211794D0709D5890707D5CA
:10292000416954F823508D60117941F0040111710F
:102930000133032BEBD130BD386A000873B51D4657
:10294000436916469A68D207044609D59A68012158
:102950009960C2F34002CDE900650021FFF768FEEF
:1029600063699A68D1050BD59A684FF480719960B4
:10297000C2F34022CDE9006501212046FFF758FE51
:1029800063699A68D2030BD59A684FF480319960D5
:10299000C2F34042CDE9006502212046FFF748FE20
:1029A000204602B0BDE87040FFF7A8BF0C4B10B541
:1029B0001C561B5C012B11D800F02AFB50EA0103C6
:1029C000024602D0421E61F10001064B53F824007A
:1029D00020B1BDE810400B46FFF7B0BF10BD00BFEF
:1029E0002C6A0008285C0020F8B5044646690029D6
:1029F0006CD106F10C07386880076AD006EB011528
:102A00003868D5F8B00110F0040FD5F8B0011ABF3E
:102A1000C00840F00040400DA061D5F8B0C11CF0E6
:102A2000020F1CBF40F08040A061D5F8B40106EB56
:102A3000011100F00F0084F82400D1F8B8012077CC
:102A4000D1F8B801000A6077D1F8B801000CA0777E
:102A5000D1F8B801000EE077D1F8BC0184F820006D
:102A6000D1F8BC01000A84F82100D1F8BC01000CA7
:102A700084F82200D1F8BC11090E84F82310382103
:102A8000396004F1340004F1180104F1240551F80F
:102A9000046B40F8046BA942F9D109880180C4E9AC
:102AA0000A2321460023238651F8283B2046DB6B6E
:102AB000984704F58052204692F8C83043F004034A
:102AC00082F8C830BDE8F840FFF718BF06F11007DC
:102AD00091E7F8BD0D4B70B51D561B5C012B0C46E4
:102AE00012D800F095FA02460B4652EA030102D0D2
:102AF000013A63F10003064951F8250020B121464F
:102B0000BDE87040FFF770BF70BD00BF2C6A0008C1
:102B1000285C0020F8B500F583511E46FFF7A8FC9D
:102B2000DFF844C00831002404F1840500EB4515AA
:102B30002B795F070ED4DB060CD5D1E900739742E1
:102B4000B34107D243695CF824709F602B7943F04E
:102B500004032B710134032C01F12001E4D1BDE801
:102B6000F840FFF78BBC00BF386A000808B5FFF7D4
:102B70007FFCFFF7C3FEBDE80840FFF77FBC000005
:102B8000F8B543690546986800F0E050B0F1E05FA1
:102B90000F461FD0E8B1FFF76BFC05F583541034E6
:102BA000002606F1840305EB43131B791A0706D5AB
:102BB0000136032E04F12004F3D1012007E05B0766
:102BC000F6D42146384600F07DFA0028F0D1FFF710
:102BD00055FCF8BD0120FCE700F5805008B5FFF773
:102BE00047FCC06DFFF726FBFFF748FC43090CBF0D
:102BF0000120002008BD0000F8B51D460023137019
:102C00000F4606461446FFF7E7FF80F001003870D4
:102C100025B129463046FFF7B3FF2070F8BD00000C
:102C20002DE9B8410C4615461F46804600F0F0F9E4
:102C30000B462178024609B9287850B14046FFF783
:102C400069FFFFF793FF3B462A462146FFF7D4FF73
:102C50000120BDE8B881000038B500F58054FFF7C9
:102C600007FC2A4D94F8C930EB5CDBB1012B27D06F
:102C7000FFF704FC94F8C830DB0746D4002944D0A1
:102C8000FFF7F6FB94F8C930EB5C33B3012B31D07E
:102C900094F8C83043F0010384F8C830BDE83840E8
:102CA000FFF7ECBB1A4B1A6C42F000721A641A6AF6
:102CB00042F000721A621A6A22F000721A62D7E7B2
:102CC000134B1A6C42F080621A641A6A42F08062F6
:102CD0001A621A6A22F08062F0E70321132001F0E1
:102CE000E5F90321142001F0E1F90321152001F099
:102CF000DDF9CDE703213F2001F0D8F90321402081
:102D000001F0D4F903214120F1E738BD286A000819
:102D1000003802402DE9F04700F5805588B095F85D
:102D2000C930022B0446884616467FD8844F57F890
:102D300023200AB947F82300D7F800A0C4F80C8074
:102D40002674BAF1000F63D095F8C930012B6FD00B
:102D500001212046FFF780FFFFF78AFB62691368B5
:102D600023F0020313606269136843F001031360E8
:102D7000636900275F6101212046FFF77FFBFFF7B2
:102D8000A7FD002800F09580E86DFFF741FA04F5F3
:102D90008359BA4609F10809202200216846FEF746
:102DA00009FF02A8FFF730FCCDF818A06A4609EB2E
:102DB00007030DF1180E9446BCE80300F4451860B3
:102DC0005960624603F10803F5D1DCF80000186091
:102DD00020379CF804201A71602FDDD195F8C83097
:102DE0006FF38203002785F8C8306A4641462046C3
:102DF000ADF80070ADF802708DF80470FFF70CFDAF
:102E0000636948BB4FF400421A6008B0BDE8F08720
:102E100041F2D00003F0F6FC814610B15146FFF7B5
:102E200097FCC7F80090B9F1000F8DD10020ECE7B6
:102E3000386803681B6B98470146002888D13868BA
:102E4000FFF70AFF3868036832465B6841469847D7
:102E500000287FF47DAFE9E761221A609DF8023017
:102E60009DF803201B06120402F4702203F0407345
:102E70001343BDF80020C2F3090213439DF8042058
:102E80001205022E02F4E0020CBF4FF000410021B7
:102E9000134362690B43D361636913225A61626908
:102EA000136823F00103136039462046FFF710FD35
:102EB00008B96369A6E795F8C930002B39D1616973
:102EC000D1F8002242F00102C1F800226169D1F874
:102ED000002222F47C5222F00E02C1F80022616925
:102EE000D1F8002242F46062C1F800226269C2F89F
:102EF00014326269C2F8043262696FF07841C2F834
:102F00000C126269C2F840326269C2F844326269E6
:102F1000C2F8B0326269C2F8B432636944F20102A5
:102F2000C3F81C226269D2F8003223F00103C2F810
:102F3000003295F8C83043F0020385F8C83064E7E2
:102F4000285C002008B50020FFF730FDBDE80840F0
:102F500001F082B808B500210846FFF7BBFDBDE8C7
:102F6000084001F079B8000008B501210020FFF702
:102F7000B1FDBDE8084001F06FB8000008B50120C0
:102F8000FFF714FDBDE8084001F066B808B5002160
:102F90000120FFF79FFDBDE8084001F05DB800008B
:102FA00008B501210846FFF795FDBDE8084001F08E
:102FB00053B8000000B59BB0EFF309816822684662
:102FC000FEF7D2FDEFF30583014B9B6BFEE700BFDD
:102FD00000ED00E008B5FFF7EDFF000000B59BB085
:102FE000EFF3098168226846FEF7BEFDEFF3058323
:102FF000014B5B6BFEE700BF00ED00E0FEE7000069
:103000000FB408B5029801F03DFDFEE702F0D4B917
:1030100002F0ACB913B56C4684E80600031D94E8D1
:10302000030083E80500012002B010BD73B5856878
:10303000019155B11B885B0707D4D0E900369B6B23
:103040009847019AC1B23046A847012002B070BD2E
:10305000F0B5866889B005460C465EB1BDF83830DB
:103060005B070AD4D0E900379B6B98472246C1B270
:103070003846B047012009B0F0BD00220023CDE959
:1030800000230023ADF808300A4603AB01F108061F
:10309000106851681C4603C40832B2422346F7D177
:1030A000106820609288A280FFF7B2FF0423ADF879
:1030B00008302B68CDE90001DB6B6946284698474C
:1030C000D8E7000030B503680968DD0FB5EBD17FA4
:1030D00023F0604421F060424FEAD1700BD0002B06
:1030E000B8BFA40C0029B8BF920C944202D034BFE0
:1030F0000120002030BD944205D1C1F38070C3F39C
:1031000080738342F6D194422CBF00200120F1E766
:103110002DE9F041456A15B94162BDE8F0814B687F
:1031200023F06047C3F38A464FEAD37EC3F3807827
:1031300016EA230638BF3E46AC462B465A68BEEB1D
:10314000D27F22F060440AD0002A18DAA40CB442DC
:1031500017D19D420FD10D60DEE71346EEE7A7427F
:1031600007D102F08044C2F3807242450BD054B1C3
:10317000EFE708D2EDE7CCF800100B60CDE7B442E2
:1031800001D0B442E5D81A689C46002AE5D11960FE
:10319000C3E700002DE9F047089D01F007044FEA5E
:1031A000D508224405F0070500EBD1004FF47F4914
:1031B000944201D1BDE8F08704F0070705F0070A43
:1031C00057453E4638BF5646C6F10806111B8E428B
:1031D00028BF0E46E10808EBD50E415C13F80EC07F
:1031E000B94029FA06F721FA0AF1FFB28CEA010187
:1031F00047FA0AF739408CEA010C03F80EC0344450
:103200003544D5E780EA0120082341F2210201B2CA
:103210004000002980B203F1FF33B8BF504013F0E3
:10322000FF03F4D17047000038B50C468D18A54255
:1032300000D138BD14F8011BFFF7E4FFF7E70000E9
:1032400042684AB1136843604389818901339BB264
:103250009942438138BF83811046704770B588B06A
:10326000202204460D4668460021FEF7A3FC2046B6
:103270000495FFF7E5FF024658B16B46054608AED8
:103280001C4603CCB44228606960234605F108055A
:10329000F6D1104608B070BD082817D909280CD0FF
:1032A0000A280CD00B280CD00C280CD00D280CD0E0
:1032B0000E2814BF4020302070470C20704710208B
:1032C0007047142070471820704720207047000076
:1032D000082817D90C280CD910280CD914280CD977
:1032E00018280CD920280CD930288CBF0F200E208C
:1032F0007047092070470A2070470B2070470C2048
:1033000070470D20704700002DE9F843078C072F08
:1033100004461ED9D0E9029800254FF6FF73C5F187
:103320002006A5F1200029FA05F108FA06F628FA88
:1033300000F031430143C9B21846FFF763FF083577
:10334000402D0346EBD1E1693A46BDE8F843FFF76B
:103350006BBF4FF6FF70BDE8F883000010B54B68F7
:1033600023B9CA8A63F30902CA8210BD04691A68C4
:103370001C600361C38A013BC3824A60EFE700001F
:103380002DE9F84F1D46CB8A0F46C3F309010529E5
:10339000814692460B4630D00020AAB207F11A04AB
:1033A0009EB2042E1FFA80F80FD8904503F1010356
:1033B00006D3FB8A0A4462F30903FB8201201AE068
:1033C0001AF80060E6540130EAE79045F1D2A1F125
:1033D000050B1C237C68BBFBF3F203FB12BB1FFA3B
:1033E0008BF6002C45D14846FFF72AFF044638B932
:1033F00078606FF00200BDE8F88F4FF00008E6E754
:10340000002606607860ADB24FF0000B454510D93C
:103410000AEB0803221D13F8011B9155B1B208F104
:1034200001081B291FFA88F82BD0454506F1010633
:10343000F1D8FB8AC3F30902154465F30903BCE71D
:10344000013292B21C462368002BF9D16B1F0B444A
:103450001C21B3FBF1F301339BB29A42D3D2BBF1EF
:10346000000FD0D14846FFF7EBFE20B9C4F800B0FA
:10347000BFE70122E7E7C0F800B05E4620600446DF
:10348000C1E74545D5D94846FFF7DAFE08B92060BF
:10349000AFE7C0F800B0002620600446B6E70000A1
:1034A0002DE9F04F2DED028B1C4683B05B69019234
:1034B00007468846002B00F09A80238C2BB1E269E6
:1034C000002A00F09480072B35D807F10C00FFF795
:1034D000B7FE054638B96FF00205284603B0BDECCB
:1034E000028BBDE8F08F14220021FEF763FB228CD3
:1034F000E16905F10800FEF737FB208C013080B24E
:10350000FFF7E6FEFFF7C8FE013880B220840130E5
:1035100028746369228C1B782A4403F01F0363F02C
:103520003F0348F000411372384669602946FFF7AF
:10353000EFFD0125D1E700F10C034FF0000908EE83
:10354000103A4FF0800A4E464D4618EE100AFFF72B
:1035500077FE83460028BED014220021FEF72AFB06
:10356000002E3AD1019BABF8083002220BF1080E75
:103570001FFA82FC0CF10100BCF1060F218C80B215
:1035800001D88E422BD3FFF7A3FEFFF785FE6269B9
:103590001278013802F01F028E4208BF4FF0400A35
:1035A00042EA49121BFA80F14AEA020A013048F065
:1035B000004281F808A08BF81000CBF8042059468F
:1035C0003846FFF7A5FD238C0135B3422DB289F0B3
:1035D00001094FF0000AB8D17FE70022C6E7E16990
:1035E000895D0EF802100136B6B20132C0E76FF005
:1035F000010572E7F8B515460E4630220021044653
:103600001F46FEF7D7FA069B6360B5F5001F079BC0
:10361000A76034BF6A094FF6FF72A36297B2E661F2
:1036200004F1100000239A4206D800230360A78209
:10363000E3822383E360F8BD066001333046203621
:10364000F1E7000003781BB94BB2002BC8BF017033
:103650007047000000787047F8B50C46C969074606
:1036600011B9238C002B37D1257E1F2D34D8387803
:1036700028BB228C072A2CD8268A36F003032BD1AC
:103680004FF6FF70FFF7D0FD20F00100310240043B
:1036900041EA0561400C41EA40254FF6FF7223469E
:1036A00029463846FFF7FCFE002807DD62691378DB
:1036B0000133DBB21F2B88BF00231370F8BD218AB2
:1036C0002D0645EA012505432046FFF71DFE02466B
:1036D000E5E76FF00300F1E76FF00100EEE70000AF
:1036E00070B58AB0044616460021282268461D4659
:1036F000FEF760FABDF83830ADF810300F9B059337
:103700009DF840308DF81830119B07936946BDF83D
:103710004830ADF820302046CDE90265FFF79CFF28
:103720000AB070BD2DE9F041D36905460C46164636
:103730000BB9138C5BBB377E1F2F28D895F8008000
:10374000B8F1000F26D03046FFF7DEFD33782102B6
:1037500041EAC33141EA0801338A41EA076141EA9B
:1037600003410246334641F080012846FFF798FEA8
:1037700000280ADD3378012B07D1726913780133F1
:10378000DBB21F2B88BF00231370BDE8F0816FF000
:103790000100FAE76FF00300F7E70000F0B58BB027
:1037A00004460D4617460021282268461E46FEF7AD
:1037B00001FA9DF84C305A1E534253418DF80030A7
:1037C0009DF84030ADF81030119B05939DF84830BE
:1037D0008DF81830149B07936A46BDF85430ADF845
:1037E000203029462046CDE90276FFF79BFF0BB03B
:1037F000F0BD0000406A00B104307047436A1A68A7
:10380000426202691A600361C38A013BC382704746
:103810002DE9F041D0F82080194E14461D4641464E
:10382000002709B9BDE8F081D1E90223A21A65EBAE
:103830000303964277EB03031ED2036A8B420DD13A
:10384000FFF78CFD036A1B68036203690B60C38A80
:103850000161016A013BC3828846E2E7FFF77EFD12
:103860000B68C8F8003003690B60C38A0161013B33
:10387000C382D8F80010D4E788460968D1E700BFB2
:1038800080841E002DE9F04F8BB00D46DDF850907E
:1038900014469B468046002800F01981B9F1000FBC
:1038A00000F01581531E3F2B00F21181012A03D134
:1038B000BBF1000F40F00B810023CDE90833B8F8CD
:1038C0001430B5EBC30F4FEAC30703D300200BB08E
:1038D000BDE8F08F2B199F42D8F80C303ABF7F1B00
:1038E000FFB227461BB9D8F81030002B7AD0272D0D
:1038F0004ED8C5F12806B7424FF000032CBFF6B2F0
:103900003E4600932946D8F8080008AB3246FFF738
:1039100041FCA7EB060A35445FFA8AFAB8F814307E
:1039200003F10053053BDB000493D8F80C300393FC
:103930002821039B13B1BAF1000F2CD1D8F8100045
:1039400040B1BAF1000F05D0009608AB5246691A93
:10395000FFF720FC38B2002FB8D066070AD00AABB8
:1039600003EBD401624211F8083C02F00702134154
:1039700001F8083C082C3CD9102C40F2B580202CD2
:1039800040F2B780BBF1000F00F09C80082334E0C8
:10399000BA460026C2E7049BE02B28BFE02306932B
:1039A0000B44AB42059314D95A1B039800969245D9
:1039B00034BF5246D2B2691A08AB04300792FFF7FF
:1039C000E9FB079A1644AAEB020A1544F6B25FFA1D
:1039D0008AFA049B069A05999B1A0493039B1B6819
:1039E0000393A6E70093D8F8080008AB3A462946A7
:1039F000AEE7BBF1000F13D00123B4EBC30F6CD0C3
:103A0000082C12D89DF82030621E23FA02F2D50746
:103A100006D54FF0FF3202FA04F423438DF820302C
:103A20009DF8203089F8003051E7102C12D8BDF8ED
:103A30002030621E23FA02F2D10706D54FF0FF3282
:103A400002FA04F42343ADF82030BDF82030A9F881
:103A500000303CE7202C0FD80899631E21FA03F3AD
:103A6000DA0705D54FF0FF3202FA04F40C4308944C
:103A7000089BC9F800302AE7402C2BD0DDE9086507
:103A8000611EC4F12102A4F1210326FA01F105FA15
:103A900002F225FA03F311431943CB0712D5012291
:103AA000A4F12003C4F1200102FA03F322FA01F188
:103AB000A240524243EA010363EB430332432B43E8
:103AC000CDE90823DDE90823C9E90023FFE66FF00B
:103AD0000100FCE66FF00800F9E6082CA0D9102CD4
:103AE000B3D9202CEED8C3E7BBF1000FADD0022331
:103AF00083E7BBF1000FBBD004237EE730B5012A7A
:103B0000144638BF0124402C85B028BF402400252E
:103B1000012ACDE9025518D81B788DF808306307C3
:103B20000AD004AB03EBD405624215F8083C02F05E
:103B30000702934005F8083C009103462246002105
:103B400002A8FFF727FB05B030BD082AE4D9102AE8
:103B500003D81B88ADF80830E1E7202A8DBFD3E9F0
:103B600000231B680293CDE90223D8E710B5CB6888
:103B70001BB98B600B618B8210BD04691A681C60D5
:103B80000361C38A013BC382CA60F0E703064CBFEE
:103B9000C0F3C0300220704708B50246FFF7F6FFB9
:103BA000022806D15306C2F30F2001D100F0030012
:103BB00008BDC2F30740FBE72DE9F04F93B0CDE914
:103BC00003230A6804461046FFF7E0FF022814BFEB
:103BD000C2F306260026002A0D46824680F2F281B4
:103BE00012F0C04940F0EE81097B002900F0EA8123
:103BF000022803D02378B34240F0E781C2F3046384
:103C00000693104602F07F030593FFF7C5FF059B5F
:103C100029444FEA834848EA0A4848EA4668CE7889
:103C200000230022CDE90823F309834648EA00086F
:103C3000029367D0059B009302466768534608A924
:103C40002046B847002800F0C381276A4FB9414693
:103C500004F10C00FFF702FB074690B96FF0020079
:103C600054E03B6998450DD03F68002FF9D141469B
:103C700004F10C00FFF7F2FA07460028EED0236AA1
:103C80003B60276297F817C006F01F08CCF3840C3E
:103C9000ACEB08001FFA80FE0028B8BF0EF1200030
:103CA000A8EB0C031FFA83FED7E90221B8BF00B2CC
:103CB000002B0793BEBF0EF120031BB2079352EAFD
:103CC000010338D0039BDFF824E39A1A049B4FF0DA
:103CD000000C63EB010196457CEB01032BD36B7B5E
:103CE00097F81AE0734519D1029B002B78D0012870
:103CF00021DC7868F8B9DFF8F0C2944570EB010375
:103D000016D337E0276A27B96FF00C0013B0BDE86F
:103D1000F08F3B699845B5D03F68F4E7B2489042D0
:103D20007CEB010301D30020F0E7029B002BFAD0CB
:103D3000079B0F2B17DCFA7DB30002F0030203F0A0
:103D40007C031343FB7539462046FFF707FB6B7B6B
:103D5000BB76029B3BB9FB7DC3F38402013262F365
:103D60008603FB75D0E76A7BBB7E9A42DBD1029B60
:103D7000002B35D0B309022B32D0039BBB60049BD0
:103D8000FB60142200210DA8FDF714FF039B0A938A
:103D9000049B0B932B1D0C932B7BADF83EB0013B8A
:103DA000DBB2ADF83C30069B8DF84230059B8DF8B8
:103DB000433094F82C308DF840A083F001038DF847
:103DC00044308DF84180A3680AA920469847FB7DBE
:103DD000C3F38403013303F01F039B02FB82A2E7BA
:103DE000FB7DC6F34012B2EBD31F40F0F480C3F367
:103DF0008403434540F0F280029A2B7BB609002AE7
:103E00004DD0F2075DD4032B40F2EB80039BBB60E7
:103E1000049BFB602B7BAE1D033BDBB23246394675
:103E200004F10C00FFF7ACFA00280CDA3946204602
:103E3000FFF794FAFB7DC3F38403013303F01F0300
:103E40009B02FB820AE7DDE90884AB883B834FF6DF
:103E5000FF73C9F12000A9F1200228FA09F104FA40
:103E600000F0014324FA02F211431846C9B2FFF7E9
:103E7000C9F909F10809B9F1400F0346E9D1B8823F
:103E80002A7B033AD2B23146FFF7CEF9FB7DB882E6
:103E9000DA43C2F3C01262F3C713FB7543E786B976
:103EA0002E1D013BDBB23246394604F10C00FFF710
:103EB00067FA0028BADB2A7BB88A013AD2B23146C7
:103EC000E2E7F98AC1F30901013B0429DAB25BD8C0
:103ED000281D002307F11B069A4208D910F801CBD0
:103EE00006F801C0013101330529DBB2F4D1039991
:103EF0000A9104990B91934207F11B010C9138BF71
:103F0000043379680D9134BF55FA83F300230E937F
:103F1000FB8AADF83EB0C3F309031A44069B8DF843
:103F20004230059B8DF8433094F82C30ADF83C209E
:103F300083F001038DF8443000238DF840A08DF804
:103F400041807B602A7BB88A013A291DFFF76CF912
:103F50003B8BB882834203D1A3680AA920469847C5
:103F600020460AA9FFF702FEFB7DBA8AC3F3840349
:103F7000013303F01F039B02FB823B8B9A420CBF71
:103F800000206FF01000C1E67B68002BAFD0052049
:103F900001E01C3033461E68002EFAD1091A081DB4
:103FA0002E1D184401EB090CBCF11B0F5FFA89F3BD
:103FB0009DD89A429BD916F8013B00F8013B09F1C4
:103FC0000109EFE76FF00900A0E66FF00A009DE637
:103FD0006FF00B009AE66FF00D0097E66FF00E00A1
:103FE00094E66FF00F0091E640420F0080841E00BF
:103FF000EFF3098305494A6B22F001024A636833F3
:1040000083F30988002383F31188704700EF00E0F1
:10401000302080F3118862B60C4B0D4AD96821F428
:10402000E0610904090C0A43DA60D3F8FC2009496D
:1040300042F08072C3F8FC200A6842F001020A6074
:104040002022DA7783F82200704700BF00ED00E0FD
:104050000003FA05001000E010B5302383F3118847
:104060000E4B5B6813F4006314D0F1EE103AEFF3DB
:104070000984683C4FF08073E361094BDB6B236676
:1040800084F3098800F0BCFC10B1064BA36110BD9D
:10409000054BFBE783F31188F9E700BF00ED00E073
:1040A00000EF00E0430600084606000800F1604308
:1040B00003F561430901C9B283F80013012200F03E
:1040C0001F039A4043099B0003F1604303F56143DA
:1040D000C3F880211A607047026843681143016089
:1040E00003B118477047000013B5446BD4F89434FB
:1040F0001A681178042915D1217C022912D1197965
:10410000128901238B4013420CD101A904F14C0008
:1041100001F0BCFFD4F89444019B21790246206849
:1041200000F0D0F902B010BD143001F03FBF000024
:104130004FF0FF33143001F039BF00004C3002F073
:1041400011B800004FF0FF334C3002F00BB8000004
:10415000143001F00DBF00004FF0FF31143001F0BA
:1041600007BF00004C3001F0DDBF00004FF0FF3210
:104170004C3001F0D7BF00000020704710B5D0F8D8
:1041800094341A6811780429044617D1017C022955
:1041900014D15979528901238B4013420ED1143026
:1041A00001F0A0FE024648B1D4F894444FF4807365
:1041B00061792068BDE8104000F072B910BD0000C0
:1041C000406BFFF7DBBF0000704700007FB5124B6C
:1041D000036000234360C0E90233012502260F4B30
:1041E000057404460290019300F18402294600966A
:1041F0004FF48073143001F051FE094B0294CDE965
:10420000006304F523724FF48073294604F14C00D7
:1042100001F018FF04B070BD8C6A0008C1410008AD
:10422000E94000080B68302282F311880A7903EB19
:10423000820290614A79093243F822008A7912B1E8
:1042400003EB820398610223C0F8941403740020E6
:1042500080F311887047000038B5037F044613B11E
:1042600090F85430ABB9201D01250221FFF734FF2F
:1042700004F1140025776FF0010100F09FFC84F831
:10428000545004F14C006FF00101BDE8384000F0DB
:1042900095BC38BD10B5012104460430FFF71CFF62
:1042A0000023237784F8543010BD000038B504464D
:1042B0000025143001F00AFE04F14C00257701F0CE
:1042C000D9FE201D84F854500121FFF705FF204638
:1042D000BDE83840FFF752BF90F8443003F0600368
:1042E000202B07D190F84520212A4FF0000303D856
:1042F0001F2A06D800207047222AFBD1C0E90E33BE
:1043000003E0034A82630722C2630364012070470B
:104310001D23002037B5D0F894341A681178042989
:1043200004461AD1017C022917D119791289012377
:104330008B40134211D100F14C05284601F05AFF81
:1043400058B101A9284601F0A1FED4F89444019B7C
:1043500021790246206800F0B5F803B030BD0000B6
:10436000F0B500EB810385B09E6904460D46FEB1B1
:10437000302383F3118804EB8507301D0821FFF7F4
:10438000ABFEFB685B691B6806F14C001BB101903A
:1043900001F08AFE019803A901F078FE024648B1B7
:1043A000039B2946204600F08DF8002383F31188F3
:1043B00005B0F0BDFB685A691268002AF5D01B8A67
:1043C000013B1340F1D104F14402EAE7093138B569
:1043D00050F82140DCB1302383F31188D4F89424C1
:1043E0001368527903EB8203DB689B695D6845B112
:1043F00004216018FFF770FE294604F1140001F053
:104400007BFD2046FFF7BAFE002383F3118838BDF9
:104410007047000001F0F0B8012303700023C0E9E9
:104420000133C36183620362C36243620363704703
:1044300038B50446302383F311880025C0E90355BD
:10444000C0E90555416001F0E7F80223237085F3C8
:104450001188284638BD000070B500EB8103054681
:104460005069DA600E46144618B110220021FDF79B
:10447000A1FBA06918B110220021FDF79BFB31467A
:104480002846BDE8704001F091B90000826802F052
:10449000011282600022C0E90422826101F012BA96
:1044A000F0B400EB81044789E4680125A4698D40DC
:1044B0003D43458123600023A2606360F0BC01F0AE
:1044C0002DBA0000F0B400EB81040789E4680125EF
:1044D00064698D403D43058123600023A2606360D1
:1044E000F0BC01F0A7BA000070B502230025044615
:1044F0000370C0E90255C0E90455C564856180F8C0
:10450000345001F0EFF863681B6823B12946204658
:10451000BDE87040184770BD0378052B10B5044600
:104520000AD080F850300523037043681B680BB134
:10453000042198470023A36010BD000001780529DD
:1045400006D190F85020436802701B6803B11847E9
:104550007047000070B590F83430044613B1002362
:1045600080F8343004F14402204601F0CDF963684C
:104570009B68B3B994F8443013F0600535D000213E
:10458000204601F06DFC0021204601F05FFC6368CD
:104590001B6813B1062120469847062384F834305F
:1045A00070BD204698470028E4D0B4F84A30E26B4A
:1045B0009A4288BFE36394F94430E56B002B4FF0D7
:1045C000300380F20381002D00F0F280092284F88C
:1045D000342083F311880021D4E90E232046FFF70D
:1045E00071FF002383F31188DAE794F8452003F084
:1045F0007F0343EA022340F20232934200F0C58077
:1046000021D8B3F5807F48D00DD8012B3FD0022BA5
:1046100000F09380002BB2D104F14C02A26302227D
:10462000E2632364C1E7B3F5817F00F09B80B3F5BB
:10463000407FA4D194F84630012BA0D1B4F84C307F
:1046400043F0020332E0B3F5006F4DD017D8B3F555
:10465000A06F31D0A3F5C063012B90D8636894F8A4
:1046600046205E6894F84710B4F848302046B047BA
:10467000002884D04368A3630368E3631AE0B3F5BA
:10468000106F36D040F6024293427FF478AF5C4B15
:10469000A3630223E3630023C3E794F84630012BAE
:1046A0007FF46DAFB4F84C3023F00203C4E90E552B
:1046B000A4F84C30256478E7B4F84430B3F5A06F23
:1046C0000ED194F8463084F84E30204601F062F85E
:1046D00063681B6813B101212046984703232370A8
:1046E0000023C4E90E339CE704F14F03A3630123C5
:1046F000C3E72378042B10D1302383F3118820469D
:10470000FFF7C4FE85F311880321636884F84F50D6
:1047100021701B680BB12046984794F84630002B57
:10472000DED084F84F300423237063681B68002BAD
:10473000D6D0022120469847D2E794F848301D068B
:1047400003F00F0120460AD501F0D0F8012804D06B
:1047500002287FF414AF2B4B9AE72B4B98E701F01C
:10476000B7F8F3E794F84630002B7FF408AF94F8DD
:10477000483013F00F01B3D01A06204602D501F0DD
:1047800083FBADE701F076FBAAE794F84630002BF7
:104790007FF4F5AE94F8483013F00F01A0D01B065B
:1047A000204602D501F05CFB9AE701F04FFB97E74A
:1047B000142284F8342083F311882B462A46294694
:1047C0002046FFF76DFE85F31188E9E65DB11522FD
:1047D00084F8342083F311880021D4E90E23204685
:1047E000FFF75EFEFDE60B2284F8342083F3118888
:1047F0002B462A4629462046FFF764FEE3E700BF22
:10480000BC6A0008B46A0008B86A000838B590F8B5
:1048100034300446002B3ED0063BDAB20F2A34D89F
:104820000F2B32D8DFE803F0373131082232313133
:104830003131313131313737C56BB0F84A309D42B3
:1048400014D2C3681B8AB5FBF3F203FB12556DB992
:10485000302383F311882B462A462946FFF732FE80
:1048600085F311880A2384F834300EE0142384F889
:104870003430302383F3118800231A46194620462A
:10488000FFF70EFE002383F3118838BD036C03B1DC
:1048900098470023E7E70021204601F0E1FA0021D4
:1048A000204601F0D3FA63681B6813B10621204645
:1048B00098470623D7E7000010B590F83430142B42
:1048C000044629D017D8062B05D001D81BB110BD3E
:1048D000093B022BFBD80021204601F0C1FA002140
:1048E000204601F0B3FA63681B6813B10621204625
:1048F0009847062319E0152BE9D10B2380F83430B3
:10490000302383F3118800231A461946FFF7DAFD96
:10491000002383F31188DAE7C3689B695B68002B87
:10492000D5D1036C03B19847002384F83430CEE727
:1049300000230375826803691B6899689142FBD262
:104940005A68036042601060586070470023037526
:10495000826803691B6899689142FBD85A680360B2
:10496000426010605860704708B50846302383F3F2
:1049700011880B7D032B05D0042B0DD02BB983F3AD
:10498000118808BD8B6900221A604FF0FF338361E4
:10499000FFF7CEFF0023F2E7D1E9003213605A603F
:1049A000F3E70000FFF7C4BF054BD9680875186826
:1049B00002681A60536001220275D860FBF72CBEB2
:1049C000385C002030B50C4BDD684B1C87B00446CA
:1049D0000FD02B46094A684600F084F92046FFF7BD
:1049E000E3FF009B13B1684600F086F9A86907B0A1
:1049F00030BDFFF7D9FFF9E7385C002069490008AE
:104A0000044B1A68DB6890689B68984294BF00204A
:104A100001207047385C0020084B10B51C68D8682E
:104A200022681A60536001222275DC60FFF78EFF56
:104A300001462046BDE81040FBF7EEBD385C002083
:104A4000044B1A68DB6892689B689A4201D9FFF7A9
:104A5000E3BF7047385C002038B5074C0749084869
:104A6000012300252370656001F0FCFB0223237005
:104A700085F3118838BD00BFA05E0020C46A00081D
:104A8000385C002008B572B6044B186500F052FC83
:104A900000F010FD024B03221A70FEE7385C002084
:104AA000A05E002000F05EB9EFF3118020B9EFF3B3
:104AB0000583302282F311887047000010B530B9A9
:104AC000EFF30584C4F3080414B180F3118810BD1A
:104AD000FFF7B6FF84F31188F9E70000034A516835
:104AE00053685B1A9842FBD8704700BF001000E083
:104AF0008B60022308618B82084670478368A3F1AC
:104B0000840243F8142C026943F8442C426943F8A8
:104B1000402C094A43F8242CC26843F8182C02227E
:104B200003F80C2C002203F80B2C044A43F8102C39
:104B3000A3F12000704700BF31060008385C002058
:104B400008B5FFF7DBFFBDE80840FFF72BBF00000B
:104B5000024BDB6898610F20FFF726BF385C00200E
:104B6000302383F31188FFF7F3BF000008B5014637
:104B7000302383F311880820FFF724FF002383F3F9
:104B8000118808BD064BDB6839B1426818605A606D
:104B9000136043600420FFF715BF4FF0FF307047EC
:104BA000385C00200368984206D01A6802605060A2
:104BB00099611846FFF7F6BE7047000038B5044605
:104BC0000D462068844200D138BD036823605C60D4
:104BD0008561FFF7E7FEF4E710B503689C68A24221
:104BE0000CD85C688A600B604C60216059609968E1
:104BF0008A1A9A604FF0FF33836010BD1B68121B46
:104C0000ECE700000A2938BF0A2170B504460D46BA
:104C10000A26601901F020FB01F00CFB041BA542E1
:104C200003D8751C2E460446F3E70A2E04D9BDE8C6
:104C30007040012001F056BB70BD0000F8B5144B68
:104C40000D46D96103F1100141600A2A1969826099
:104C500038BF0A22016048601861A818144601F0A4
:104C6000EDFA0A2701F0E6FA431BA342064606D3F3
:104C70007C1C281901F0F0FA27463546F2E70A2F86
:104C800004D9BDE8F840012001F02CBBF8BD00BFFD
:104C9000385C0020F8B506460D4601F0CBFA0F4A05
:104CA000134653F8107F9F4206D12A4601463046EC
:104CB000BDE8F840FFF7C2BFD169BB68441A2C19A0
:104CC00028BF2C46A34202D92946FFF79BFF224664
:104CD00031460348BDE8F840FFF77EBF385C00204E
:104CE000485C002010B4C0E9032300235DF8044BA6
:104CF0004361FFF7CFBF000010B5194C23699842FC
:104D00000DD0D0E90032816813605A609A680A4475
:104D10009A60002303604FF0FF33A36110BD234668
:104D2000026843F8102F53600022026022699A4201
:104D300003D1BDE8104001F089BA936881680B4443
:104D4000936001F077FA2269E1699268441AA242FD
:104D5000E4D91144BDE81040091AFFF753BF00BF62
:104D6000385C00202DE9F047DFF8BC8008F110071F
:104D70002C4ED8F8105001F05DFAD8F81C40AA6803
:104D8000031B9A423ED81444D5E900324FF0000983
:104D9000C8F81C4013605A60C5F80090D8F810306D
:104DA000B34201D101F052FA89F31188D5E90331F8
:104DB00028469847302383F311886B69002BD8D09D
:104DC00001F038FA6A69A0EB04094A4582460DD21F
:104DD000022001F087FA0022D8F81030B34208D13F
:104DE00051462846BDE8F047FFF728BF121A224473
:104DF000F2E712EB090938BF4A4629463846FFF761
:104E0000EBFEB5E7D8F81030B34208D01444211AAD
:104E1000C8F81C00A960BDE8F047FFF7F3BEBDE885
:104E2000F08700BF485C0020385C002000207047FD
:104E3000FEE70000704700004FF0FF3070470000B1
:104E400002290CD0032904D00129074818BF0020EB
:104E50007047032A05D8054800EBC2007047044894
:104E600070470020704700BF9C6B00082C23002077
:104E7000506B000870B59AB00546084601A9144663
:104E800000F0C2F801A8FCF78DFE431C5B00C5E9E9
:104E900000340022237003236370C6B201AB0234D6
:104EA0001046D1B28E4204F1020401D81AB070BD8E
:104EB00013F8011B04F8021C04F8010C0132F0E79E
:104EC00008B5302383F311880348FFF723FA002342
:104ED00083F3118808BD00BFA85E002090F844301D
:104EE00003F01F02012A07D190F845200B2A03D1B5
:104EF0000023C0E90E3315E003F06003202B08D136
:104F0000B0F848302BB990F84520212A03D81F2A41
:104F100004D8FFF7E1B9222AEBD0FAE7034A82630B
:104F20000722C26303640120704700BF24230020CE
:104F300007B5052917D8DFE801F01916031919205C
:104F4000302383F31188104A01900121FFF784FA7E
:104F500001980E4A0221FFF77FFA0D48FFF7A6F9E4
:104F6000002383F3118803B05DF804FB302383F33F
:104F700011880748FFF770F9F2E7302383F31188AF
:104F80000348FFF787F9EBE7F06A0008146B0008A5
:104F9000A85E002038B50C4D0C4C0D492A4604F192
:104FA0000800FFF767FF05F1CA0204F11000094984
:104FB000FFF760FF05F5CA7204F118000649BDE865
:104FC0003840FFF757BF00BF706300202C2300203C
:104FD000D06A0008DA6A0008E56A000870B504467D
:104FE00008460D46FCF7DEFDC6B2204601340378C4
:104FF0000BB9184670BD32462946FCF7BFFD0028A4
:10500000F3D10120F6E700002DE9F84F05460C46E4
:10501000FCF7C8FD2B49C6B22846FFF7DFFF08B1F1
:105020000536F6B228492846FFF7D8FF08B11036F2
:10503000F6B2632E0DD8DFF88C80DFF88C90234F0A
:10504000DFF890A0DFF890B02E7846B92670BDE862
:10505000F88F29462046BDE8F84F01F091BC252E77
:105060002BD1072241462846FCF788FD58B9DBF8CA
:1050700000302360DBF804306360DBF80830A360A5
:1050800007350C34E0E7082249462846FCF776FD50
:1050900098B90F4BA21C197809090232C95D02F8B0
:1050A000041C13F8011B01F00F015345C95D02F800
:1050B000031CF0D118340835C6E704F8016B01353C
:1050C000C2E700BFBC6B0008E56A0008D16B0008AE
:1050D000107AFF1F1C7AFF1FC46B0008BFF34F8FAD
:1050E000024AD368DB03FCD4704700BF003C024097
:1050F00008B5094B1B7873B9FFF7F0FF074B1A6926
:10510000002ABFBF064A5A6002F188325A601A6804
:1051100022F480621A6008BDCE650020003C024087
:105120002301674508B50B4B1B7893B9FFF7D6FFF2
:10513000094B1A6942F000421A611A6842F480521F
:105140001A601A6822F480521A601A6842F4806267
:105150001A6008BDCE650020003C02400728F0B56B
:1051600016D80C4C0C4923787BB90C4D0E460823FD
:105170004FF0006255F8047B46F8042B013B13F016
:10518000FF033A44F6D10123237051F82000F0BD0B
:105190000020FCE7F0650020D0650020E46B0008EB
:1051A000014B53F820007047E46B0008082070475B
:1051B000072810B5044601D9002010BDFFF7CEFF27
:1051C000064B53F824301844C21A0BB90120F4E7F7
:1051D00012680132F0D1043BF6E700BFE46B00082F
:1051E000072810B5044621D8FFF778FFFFF780FFA6
:1051F0000F4AF323D360C300DBB243F4007343F0E0
:1052000002031361136943F480331361FFF766FFF0
:10521000FFF7A4FF074B53F8241000F047F9FFF7FE
:1052200081FF2046BDE81040FFF7C2BF002010BD3F
:10523000003C0240E46B0008F8B512F0010314468C
:1052400042D185182E4A954257D82E4B1B6813F031
:10525000010352D02C4DFFF74BFFF323EB60FFF718
:105260003DFF40F20127032C15D824F001046618F5
:10527000254C401A40F20117B142236900EB0105A9
:1052800024D123F001032361FFF74CFF0120F8BD77
:10529000043C0430E7E78307E7D12B6923F440732C
:1052A0002B612B693B432B6151F8046B0660BFF304
:1052B0004F8FFFF713FF03689E42E9D02B6923F05D
:1052C00001032B61FFF72EFF0020E0E723F440737A
:1052D000236123693B4323610B882B80BFF34F8FEE
:1052E000FFF7FCFE2D8831F8023BADB2AB42C3D0D4
:1052F000236923F001032361E4E71846C7E700BFF1
:105300000000080800380240003C0240084908B587
:105310000B7828B11BB9FFF7EBFE01230B7008BD1A
:10532000002BFCD0BDE808400870FFF7FBBE00BFB3
:10533000CE65002008B54FF400314FF0005000F06A
:10534000B7F8BDE808404FF480314FF0805000F0CE
:10535000AFB800000846114601F076BA012001F00E
:1053600073BA0000084601F08DBA000070B582B033
:10537000FFF79AFB0E4E054600F05CFF3268904244
:1053800037BF0C4A0B49516814682EBFD1E9004160
:10539000013151600419034641F100012846019191
:1053A0003360FFF78BFB0199204602B070BD00BF50
:1053B000F4650020F865002070B582B0FFF774FB3B
:1053C000104E054600F036FF3268904237BF0E4A55
:1053D0000D49516814682EBFD1E900410131516077
:1053E000041941F100010346284601913360FFF79B
:1053F00065FB01994FF47A7200232046FAF7F8FE14
:1054000002B070BDF4650020F865002010B50244BC
:10541000064BD2B2904200D110BD441C00B253F8EA
:10542000200041F8040BE0B2F4E700BF5028004030
:105430000F4B30B51C6F240407D41C6F44F4007468
:105440001C671C6F44F400441C670A4C236843F437
:10545000807323600244084BD2B2904200D130BD29
:10546000441C00B251F8045B43F82050E0B2F4E76A
:1054700000380240007000405028004007B501226B
:1054800001A90020FFF7C2FF019803B05DF804FBFB
:1054900013B50446FFF7F2FFA04205D0012201A98F
:1054A00000200194FFF7C4FF02B010BD7047000058
:1054B0007047000070470000074B45F255521A60D4
:1054C00002225A6040F6FF729A604CF6CC421A6093
:1054D000024B01221A707047003000400466002021
:1054E000034B1B781BB1034B4AF6AA221A60704784
:1054F0000466002000300040034B1A681AB9034AC2
:10550000D2F874281A60704700660020003002400C
:10551000024B4FF08072C3F874287047003002408D
:1055200008B5FFF7E9FF024B1868C0F3407008BDEB
:105530000066002008B5FFF7DFFF024B1868C0F3D4
:10554000007008BD0066002070470000FEE7000004
:105550000A4B0B480B4A90420BD30B4BDA1C121A26
:10556000C11E22F003028B4238BF00220021FCF74B
:1055700021BB53F8041B40F8041BECE7F86D00084E
:1055800008670020086700200867002070B5D0E990
:1055900015439E6800224FF0FF3504EB4213510182
:1055A000D3F800090028BEBFD3F8000940F08040BE
:1055B000C3F80009D3F8000B0028BEBFD3F8000BD6
:1055C00040F08040C3F8000B013263189642C3F8E4
:1055D0000859C3F8085BE0D24FF00113C4F81C3837
:1055E00070BD0000890141F02001016103699B0643
:1055F000FCD41220FFF772BA10B5054C2046FEF716
:105600000BFF4FF0A0436365024BA36510BD00BFC5
:1056100008660020286C000870B50378012B054649
:1056200050D12A4B446D98421BD1294B5A6B42F002
:1056300080025A635A6D42F080025A655A6D5A6967
:1056400042F080025A615A6922F080025A610E21AA
:1056500043205B69FEF72AFD1E4BE3601E4BC4F836
:1056600000380023C4F8003EC02323606E6D4FF461
:105670000413A3633369002BFCDA012333610C208C
:10568000FFF72CFA3369DB07FCD41220FFF726FA68
:105690003369002BFCDA0026A6602846FFF776FF68
:1056A0006B68C4F81068DB68C4F81468C4F81C6838
:1056B0004BB90A4BA3614FF0FF336361A36843F01A
:1056C0000103A36070BD064BF4E700BF086600202D
:1056D000003802404014004003002002003C30C06B
:1056E000083C30C0F8B5446D054600212046FFF760
:1056F00079FFA96D00234FF001128F68C4F8343888
:105700004FF00066C4F81C284FF0FF3004EB431242
:1057100001339F42C2F80069C2F8006BC2F8080961
:10572000C2F8080BF2D20B686A6DEB656362102356
:105730001361166916F01006FBD11220FFF7CEF99F
:10574000D4F8003823F4FE63C4F80038A36943F4A6
:10575000402343F01003A3610923C4F81038C4F8B0
:1057600014380A4BEB604FF0C043C4F8103B084BB1
:10577000C4F8003BC4F81069C4F80039EB6D03F1BC
:10578000100243F48013EA65A362F8BD046C0008BC
:1057900040800010426D90F84E10D2F8003823F48B
:1057A000FE6343EA0113C2F8003870472DE9F8435D
:1057B00000EB8103456DDA68166806F00306731E78
:1057C000022B05EB41130C4680460FFA81F94FEA94
:1057D00041104FF00001C3F8101B4FF0010104F11C
:1057E000100398BFB60401FA03F391698EBF334EDC
:1057F00006F1805606F5004600293AD0578A04F192
:105800005801490137436F50D5F81C180B43C5F8B0
:105810001C382B180021C3F8101953690127611E89
:10582000A7409BB3138A928B9B08012A88BF5343DE
:10583000D8F85C20981842EA034301F1400205EBD6
:105840008202C8F85C00214653602846FFF7CAFE72
:1058500008EB8900C3681B8A43EA84534834640117
:105860001E432E51D5F81C381F43C5F81C78BDE8DF
:10587000F88305EB4917D7F8001B21F40041C7F85E
:10588000001BD5F81C1821EA0303C0E704F13F030D
:1058900005EB83030A4A5A6028462146FFF7A2FE19
:1058A00005EB4910D0F8003923F40043C0F8003963
:1058B000D5F81C3823EA0707D7E700BF008000109F
:1058C00000040002826D1268C265FFF75FBE00002F
:1058D0005831436D49015B5813F4004004D013F470
:1058E000001F0CBF02200120704700004831436DAB
:1058F00049015B5813F4004004D013F4001F0CBF9F
:10590000022001207047000000EB8101CB68196A7A
:105910000B6813604B6853607047000000EB810315
:1059200030B5DD68AA691368D36019B9402B84BF0C
:10593000402313606B8A1468426D1C44013CB4FB25
:10594000F3F46343033323F0030302EB411043EA10
:10595000C44343F0C043C0F8103B2B6803F003037B
:10596000012B09B20ED1D2F8083802EB411013F422
:10597000807FD0F8003B14BF43F0805343F00053C6
:10598000C0F8003B02EB4112D2F8003B43F0044365
:10599000C2F8003B30BD00002DE9F041244D6E6D92
:1059A00006EB40130446D3F8087BC3F8087B38079E
:1059B0000AD5D6F81438190706D505EB8403214615
:1059C000DB6828465B689847FA071FD5D6F8143875
:1059D000DB071BD505EB8403D968CCB98B69488AF2
:1059E0005A68B2FBF0F600FB16228AB91868DA682A
:1059F00090420DD2121AC3E90024302383F3118898
:105A00000B482146FFF78AFF84F31188BDE8F08137
:105A1000012303FA04F26B8923EA02036B81CB684A
:105A2000002BF3D021460248BDE8F041184700BFE3
:105A30000866002000EB810370B5DD68436D6C697A
:105A40002668E6604A0156BB1A444FF40020C2F8AB
:105A500010092A6802F00302012A0AB20ED1D3F813
:105A6000080803EB421410F4807FD4F8000914BF37
:105A700040F0805040F00050C4F8000903EB42129F
:105A8000D2F8000940F00440C2F80009D3F8340805
:105A9000012202FA01F10143C3F8341870BD19B9AB
:105AA000402E84BF4020206020682E8A8419013C4B
:105AB000B4FBF6F440EAC44040F000501A44C6E794
:105AC0002DE9F8433B4D6E6D06EB40130446D3F8C9
:105AD0000889C3F8088918F0010F4FEA40171AD057
:105AE000D6F81038DB0716D505EB8003D9684B696B
:105AF0001868DA68904230D2121A4FF000091A6022
:105B0000C3F80490302383F3118821462846FFF719
:105B100091FF89F3118818F0800F1CD0D6F8343823
:105B20000126A640334216D005EB84036D6DD3F8F1
:105B30000CC0DCF814200134E4B2D2F800E005EB2C
:105B400004342F445168714515D3D5F8343823EA0D
:105B50000606C5F83468BDE8F883012303FA04F2A9
:105B60002B8923EA02032B818B68002BD3D021469B
:105B700028469847CFE7BCF81000AEEB01038342FC
:105B800028BF0346D7F8180980B2B3EB800FE2D8DC
:105B90009068A0F1040959F8048FC4F80080A0EBC4
:105BA00009089844B8F1040FF5D818440B449060E4
:105BB0005360C7E7086600202DE9F74FA24C656DDA
:105BC0006E69AB691E4016F480586E6107D020469E
:105BD000FEF78AFC03B0BDE8F04FFEF73DBA002E99
:105BE00012DAD5F8003E98489B071EBFD5F8003E54
:105BF00023F00303C5F8003ED5F8043823F0010371
:105C0000C5F80438FEF79AFC370505D58E48FFF72E
:105C1000BDFC8D48FEF780FCB0040CD5D5F80838E3
:105C200013F0060FEB6823F470530CBF43F41053CA
:105C300043F4A053EB6031071BD56368DB681BB9E5
:105C4000AB6923F00803AB612378052B0CD1D5F8A1
:105C5000003E7D489A071EBFD5F8003E23F003039F
:105C6000C5F8003EFEF76AFC6368DB680BB1764856
:105C70009847F30274D4B70227D5D4F85490DFF8CC
:105C8000C8B100274FF0010A09EB4712D2F8003BD8
:105C900003F44023B3F5802F11D1D2F8003B002B41
:105CA0000DDA62890AFA07F322EA0303638104EB3F
:105CB0008703DB68DB6813B1394658469847A36D04
:105CC00001379B68FFB29F42DED9F00617D5676D9A
:105CD0003A6AC2F30A1002F00F0302F4F012B2F5AE
:105CE000802F00F08580B2F5402F08D104EB8303AC
:105CF0000022DB681B6A07F5805790426AD13003A7
:105D0000D5F8184813D5E10302D50020FFF744FE6B
:105D1000A20302D50120FFF73FFE630302D5022054
:105D2000FFF73AFE270302D50320FFF735FE750380
:105D30007FF550AFE00702D50020FFF7C1FEA107B5
:105D400002D50120FFF7BCFE620702D50220FFF753
:105D5000B7FE23077FF53EAF0320FFF7B1FE39E71B
:105D6000636DDFF8E4A0019300274FF00109A36DF4
:105D70009B685FFA87FB9B453FF67DAF019B03EB7A
:105D80004B13D3F8001901F44021B1F5802F1FD136
:105D9000D3F8001900291BDAD3F8001941F090411B
:105DA000C3F80019D3F800190029FBDB5946606DD0
:105DB000FFF718FC218909FA0BF321EA0303238179
:105DC00004EB8B03DB689B6813B159465046984738
:105DD0000137CCE7910708BFD7F80080072A98BFA2
:105DE00003F8018B02F1010298BF4FEA182884E7FB
:105DF000023304EB830207F580575268D2F818C0CB
:105E0000DCF80820DCE9001CA1EB0C0C0021884226
:105E10000AD104EB830463689B699A6802449A6020
:105E20005A6802445A606AE711F0030F08BFD7F8B6
:105E300000808C4588BF02F8018B01F1010188BF09
:105E40004FEA1828E3E700BF08660020436D03EB24
:105E50004111D1F8003B43F40013C1F8003B7047F7
:105E6000436D03EB4111D1F8003943F40013C1F83D
:105E700000397047436D03EB4111D1F8003B23F427
:105E80000013C1F8003B7047436D03EB4111D1F89B
:105E9000003923F40013C1F80039704730B5039C72
:105EA0000172043304FB0325C0E90653049B03631A
:105EB0000021059BC160C0E90000C0E90422C0E9DF
:105EC0000842C0E90A11436330BD0000416A002264
:105ED000C0E90411C0E90A22C2606FF00101FEF7B7
:105EE0006DBE0000D0E90432934201D1C2680AB904
:105EF000181D70470020704703691960C26801329D
:105F0000C260C269134482690361934224BF436A39
:105F100003610021FEF746BE38B504460D46E3682E
:105F20003BB16269131D1268A3621344E36200204F
:105F300007E0237A33B929462046FEF723FE0028DE
:105F4000EDDA38BD6FF00100FBE70000C368C269FD
:105F5000013BC3604369134482694361934224BF98
:105F6000436A436100238362036B03B118477047A0
:105F700070B53023044683F31188866A3EB9FFF773
:105F8000CBFF054618B186F31188284670BDA36A79
:105F9000E26A13F8015BA362934202D32046FFF743
:105FA000D5FF002383F31188EFE700002DE9F84FB8
:105FB00004460E46174698464FF0300989F311887B
:105FC0000025AA46D4F828B0BBF1000F09D14146FC
:105FD0002046FFF7A1FF20B18BF311882846BDE8CA
:105FE000F88FD4E90A12A7EB050B521A934528BF84
:105FF0009346BBF1400F1BD9334601F1400251F8E3
:10600000040B43F8040B9142F9D1A36A40334036A4
:10601000A3624035D4E90A239A4202D32046FFF70F
:1060200095FF8AF31188BD42D8D289F31188C9E758
:1060300030465A46FBF798FDA36A5B445E44A36270
:106040005D44E7E710B5029C0172043303FB0421B1
:10605000C0E906130023C0E90A33039B0363049BD2
:10606000C460C0E90000C0E90422C0E908424363FB
:1060700010BD0000026AC260426AC0E90422002228
:10608000C0E90A226FF00101FEF798BDD0E90423B0
:106090009A4201D1C26822B9184650F8043B0B60FD
:1060A000704700231846FAE7C368C2690133C3602A
:1060B0004369134482694361934224BF436A436145
:1060C0000021FEF76FBD000038B504460D46E368B9
:1060D0003BB123691A1DA262E2691344E362002006
:1060E00007E0237A33B929462046FEF74BFD002806
:1060F000EDDA38BD6FF00100FBE7000003691960BD
:10610000C268013AC260C269134482690361934262
:1061100024BF436A036100238362036B03B1184702
:106120007047000070B530230D460446114683F3D6
:106130001188866A2EB9FFF7C7FF10B186F3118860
:1061400070BDA36A1D70A36AE26A01339342A36221
:1061500004D3E16920460439FFF7D0FF002080F323
:106160001188EDE72DE9F84F04460D469046994613
:106170004FF0300A8AF311880026B346A76A4FB958
:1061800049462046FFF7A0FF20B187F3118830462B
:10619000BDE8F88FD4E90A073A1AA8EB0607974238
:1061A00028BF1746402F1BD905F1400355F8042B93
:1061B00040F8042B9D42F9D1A36A4033A3624036D4
:1061C000D4E90A239A4204D3E16920460439FFF74F
:1061D00095FF8BF311884645D9D28AF31188CDE714
:1061E00029463A46FBF7C0FCA36A3B443D44A36200
:1061F0003E44E5E7D0E904239A4217D1C3689BB136
:10620000836A8BB1043B9B1A0ED01360C368013BB9
:10621000C360C3691A44836902619A4224BF436A16
:106220000361002383620123184670470023FBE7C4
:1062300000F0D2B84FF08043586A70474FF0804367
:10624000002258631A610222DA6070474FF08043DF
:106250000022DA60704700004FF0804358637047B7
:10626000FEE7000070B51B4B01630025044686B0B5
:10627000586085620E46FDF7CBFE04F11003C4E9B9
:1062800004334FF0FF33C4E90635C4E90044A56088
:10629000E562FFF7CFFF2B460246C4E9082304F16D
:1062A00034010D4A256580232046FEF721FC012399
:1062B000E0600A4A0375009272680192B268CDE903
:1062C0000223074B6846CDE90435FEF739FC06B0DA
:1062D00070BD00BFA05E0020346C0008396C00085F
:1062E00061620008024AD36A1843D062704700BF57
:1062F000385C00204B6843608B688360CB68C36068
:106300000B6943614B6903628B6943620B680360ED
:106310007047000008B5264B26481A6940F2FF1165
:106320000A431A611A6922F4FF7222F001021A610B
:106330001A691A6B0A431A631A6D0A431A651E4AD0
:106340001B6D1146FFF7D6FF02F11C0100F58060BE
:10635000FFF7D0FF02F1380100F58060FFF7CAFFB8
:1063600002F1540100F58060FFF7C4FF02F17001F3
:1063700000F58060FFF7BEFF02F18C0100F5806040
:10638000FFF7B8FF02F1A80100F58060FFF7B2FF48
:1063900002F1C40100F58060FFF7ACFF02F1E001FB
:1063A00000F58060FFF7A6FFBDE8084000F090B858
:1063B0000038024000000240406C000808B500F0C0
:1063C000FBF9FEF749FBFFF797F8BDE80840FEF739
:1063D000E1BD0000704700000F4B1A6C42F0010253
:1063E0001A641A6E42F001021A660C4A1B6E936818
:1063F00043F0010393604FF0804353229A624FF0C1
:10640000FF32DA6200229A615A63DA605A6001222E
:106410005A611A60704700BF00380240002004E053
:106420004FF0804208B51169D3680B40D9B2C94317
:106430009B07116107D5302383F31188FEF732FBE8
:10644000002383F3118808BD1F4B1A696FEAC252FB
:106450006FEAD2521A611A69C2F308021A614FF048
:10646000FF301A695A69586100215A6959615A699D
:106470001A6A62F080521A621A6A02F080521A6234
:106480001A6A5A6A58625A6A59625A6A1A6C42F00F
:1064900080521A641A6E42F080521A661A6E0B4AC3
:1064A000106840F480701060186F00F44070B0F510
:1064B000007F1EBF4FF4803018671967536823F4BC
:1064C0000073536000F054B900380240007000407F
:1064D000334B4FF080521A64324A4FF440411160FE
:1064E0001A6842F001021A601A689107FCD59A688E
:1064F00022F003029A602A4B9A6812F00C02FBD138
:10650000196801F0F90119609A601A6842F4803242
:106510001A601A689203FCD55A6F42F001025A675A
:106520001F4B5A6F9007FCD51F4A5A601A6842F0F9
:1065300080721A601B4A53685904FCD5184B1A68BC
:106540009201FCD5194A9A60194B1A68194B9A4264
:10655000194B21D1194A1168194A91421CD140F2B4
:1065600005121A60144A136803F00F03052BFAD1C1
:106570000B4B9A6842F002029A609A6802F00C0291
:10658000082AFAD15A6C42F480425A645A6E42F494
:1065900080425A665B6E704740F20572E1E700BFC9
:1065A00000380240007000400854400700948838CA
:1065B000002004E011640020003C024000ED00E0F7
:1065C00041C20F41074A08B5536903F00103536103
:1065D00023B1054A13680BB150689847BDE80840DD
:1065E000FDF73ABD003C014080660020074A08B52F
:1065F000536903F00203536123B1054A93680BB159
:10660000D0689847BDE80840FDF726BD003C014032
:1066100080660020074A08B5536903F004035361FC
:1066200023B1054A13690BB150699847BDE808408A
:10663000FDF712BD003C014080660020074A08B506
:10664000536903F00803536123B1054A93690BB101
:10665000D0699847BDE80840FDF7FEBC003C01400A
:1066600080660020074A08B5536903F010035361A0
:1066700023B1054A136A0BB1506A9847BDE8084038
:10668000FDF7EABC003C014080660020164B10B5C7
:106690005C6904F478725A61A30604D5134A936ABC
:1066A0000BB1D06A9847600604D5104A136B0BB142
:1066B000506B9847210604D50C4A936B0BB1D06BF5
:1066C0009847E20504D5094A136C0BB1506C984702
:1066D000A30504D5054A936C0BB1D06C9847BDE86F
:1066E0001040FDF7B9BC00BF003C014080660020AF
:1066F000194B10B55C6904F47C425A61620504D5FB
:10670000164A136D0BB1506D9847230504D5134AF3
:10671000936D0BB1D06D9847E00404D50F4A136E0A
:106720000BB1506E9847A10404D50C4A936E0BB17F
:10673000D06E9847620404D5084A136F0BB1506FAE
:106740009847230404D5054A936F0BB1D06F98473F
:10675000BDE81040FDF780BC003C01408066002091
:1067600008B5FFF75DFEBDE80840FDF775BC000009
:10677000062108B50846FDF799FC06210720FDF71C
:1067800095FC06210820FDF791FC06210920FDF764
:106790008DFC06210A20FDF789FC06211720FDF754
:1067A00085FC06212820FDF781FCBDE80840072173
:1067B0001C20FDF77BBC000008B5FFF745FE00F08C
:1067C0000BF8FDF727FEFDF7FFFCFFF703FEBDE822
:1067D0000840FFF72DBD00000023054A194601338C
:1067E000102BC2E9001102F10802F8D1704700BF76
:1067F000806600200B460146184600F02DB80000C8
:1068000000F040B8012838BF012010B504462046EA
:1068100000F030F830B900F007F808B900F00CF8D3
:106820008047F4E710BD0000024B1868BFF35B8F90
:10683000704700BF0067002008B5062000F084F80C
:106840000120FEF7F5FA0000024B0A4601461868DF
:10685000FEF780BD4C23002010B5054C13462CB12B
:106860000A4601460220AFF3008010BD2046FCE737
:1068700000000000024B01461868FEF76FBD00BF24
:106880004C230020024B01461868FEF76BBD00BF89
:106890004C23002010B501390244904201D1002060
:1068A00005E0037811F8014FA34201D0181B10BD79
:1068B0000130F2E72DE9F041A3B1C91A177801447C
:1068C000044603F1FF3C8C42204601D9002009E038
:1068D0000578BD4204F10104F5D10CEB0405D6188E
:1068E000A54201D1BDE8F08115F8018D16F801ED42
:1068F000F045F5D0E7E700001F2938B504460D46FE
:1069000004D9162303604FF0FF3038BD426C12B13A
:1069100052F821304BB9204600F030F82A460146A3
:106920002046BDE8384000F017B8012B0AD0591CAA
:1069300003D1162303600120E7E7002442F8254035
:10694000284698470020E0E7024B01461868FFF709
:10695000D3BF00BF4C23002038B5074D00230446A9
:10696000084611462B60FEF767FA431C02D12B68DC
:1069700003B1236038BD00BF04670020FEF756BA9C
:10698000034611F8012B03F8012B002AF9D17047B7
:1069900073772D737061722D663430372D626C0001
:1069A00053544D3332463F3F3F0053544D333246EC
:1069B0003430780053544D333246343278005354D7
:1069C0004D3332463434365858000000012033002D
:1069D0000010410001105A00031059000710310047
:1069E00000000000A069000813040000AA69000864
:1069F00019040000B469000821040000BE69000801
:106A000040A2E4F1646891060041A3E5F265699251
:106A1000070000004261642043414E49666163659E
:106A200020696E6465782E00000100000001FF00FF
:106A3000006400400068004080000000008000000A
:106A40000000800000000000000000008924000811
:106A5000152D0008212C000899240008CD240008D9
:106A6000C92600089D240008AD240008A1240008C0
:106A7000A9240008A5240008F1250008B124000875
:106A800015300008C1240008C525000800000000DA
:106A900045410008314100086D4100085941000896
:106AA00065410008514100083D41000829410008A6
:106AB0007941000800000000010000000000000013
:106AC00063300000C06A0008905C0020A05E0020D7
:106AD0004172647550696C6F740025424F41524495
:106AE000252D424C002553455249414C25000000BC
:106AF000020000000000000061430008CD430008D0
:106B0000400040004063002050630020020000006D
:106B10000000000003000000000000001144000815
:106B20000000000010000000606300200000000072
:106B300001000000000000000866002001010200C2
:106B4000314F0008414E0008DD4E0008C14E0008DC
:106B500043000000586B000809024300020100C016
:106B600032090400000102020100052400100105A1
:106B70002401000104240202052406000107058205
:106B8000030800FF09040100020A000000070501D4
:106B900002400000070581024000000012000000D2
:106BA000A46B0008120110010200004009124157B5
:106BB00000020102030100000403090425424F41C1
:106BC0005244250073772D737061722D663430370F
:106BD0000030313233343536373839414243444559
:106BE000460000000040000000400000004000009F
:106BF0000040000000000100000002000000020050
:106C00000000020000000000554500080D48000883
:106C1000B94800084000400068660020686600200F
:106C200001000000786600208000000040010000A4
:106C3000030000006D61696E0069646C650000000E
:106C40000000802A00000000AAAAAAAA00000024CE
:106C5000FFFF00000000000000A00A000068000024
:106C600000000000AA6AAAAA000000007FFF00003E
:106C7000000090090000000000000100000000007A
:106C8000AAAAAAAA00000000FFFE0000000000005F
:106C9000000000001A000000000000009AAAAAAA42
:106CA00000000000FFFF000099000000000000004D
:106CB0000000000000000000AAAAAAAA000000002C
:106CC000FFFF0000000000000000000000000000C6
:106CD00000000000AAAAAAAA00000000FFFF00000E
:106CE00000000000000000000000000000000000A4
:106CF000AAAAAAAA00000000FFFF000000000000EE
:106D00000000000000000000000000000A00000079
:106D10000000000003000000000000000000000070
:106D20000000000000000000000000000000000063
:106D3000000000000000000000000000E494FF7F5D
:106D400001000000000000007017000000000000BB
:106D5000000007000000000040420F00FE2A010072
:106D6000D2040000FF00960000000008009600001A
:106D70000000080004000000B86B000800000000DC
:106D80000000000000000000000000000000000003
:106D90000000000050230020000000000000000060
:106DA00000000000000000000000000000000000E3
:106DB00000000000000000000000000000000000D3
:106DC00000000000000000000000000000000000C3
:106DD00000000000000000000000000000000000B3
:106DE00000000000000000000000000000000000A3
:086DF00000000000000000009B
:00000001FF
